:020000040800F2
:10700000602C0020017100081D7C00080D7B000829
:10701000197C0008A7750008CD8E0008000000004C
:10702000000000000000000000000000397E0008A1
:107030004D77000800000000177100081971000862
:107040001B7100081B7100081B7100081B710008F0
:107050001B7100081B7100081B7100081B710008E0
:107060001B7100081B7100081B7100081B710008D0
:107070001B7100081B7100081B7100081B710008C0
:107080001B7100081B7100081B7100081B710008B0
:107090001B7100081B7100081B7100081B710008A0
:1070A0001B7100081B7100081B7100081B71000890
:1070B000ED810008D1830008518500081B7100088C
:1070C0001B7100081B7100081B7100081B71000870
:1070D0001B7100080D8D00081B7100081B71000852
:1070E0001B7100081B7100081B710008DFF80CD031
:1070F00000F046F9004800474DB10008602C002020
:107100000648804706480047FEE7FEE7FEE7FEE741
:10711000FEE7FEE7FEE7FEE7FEE7FEE74D7F00083D
:10712000ED70000840EA01039B0703D009E008C99D
:10713000121F08C0042AFAD203E011F8013B00F83C
:10714000013B521EF9D270472DE9FE4F81EA03043C
:1071500004F0004421F0004100944FF0000B23F0B4
:10716000004350EA01045ED052EA03045BD0C3F34B
:107170000A54C1F30A552C44A4F2F3340194A0FB41
:107180000254C1F3130141F48011C3F3130343F418
:10719000801301FB024400FB034E840A970A44EA71
:1071A000815447EA8357A4FB076802958D0A05FBC3
:1071B00007854FEA932C04FB0C542705029D4FEAE8
:1071C000065847EA1637B5EB08056EEB070C870E35
:1071D000920E47EA811742EA8312A7FB0201B6EB3F
:1071E0000B0164EB00042B0D43EA0C335E1844EBF7
:1071F0001C50DA465146E7FB0201C5F313044FEA7F
:107200000B3343EA14534FEA0432019C43EA06036A
:10721000A4F10C040294009CCDE900B400F061F8E4
:1072200003B0BDE8F08F00200146F9E70EB540F24B
:10723000334102910021CDE900110A460B4600F0CE
:1072400050F803B000BDC1F30A5210B5C1F31301E9
:1072500040F2FF3341F480119A4201DA002010BD60
:1072600040F233439A42A2F2334203DC524200F02E
:1072700019F810BD904010BD30B50B4601460020F6
:107280002022012409E021FA02F59D4205D303FAE8
:1072900002F5491B04FA02F52844151EA2F1010269
:1072A000F1DC30BD202A04DB203A21FA02F0002173
:1072B000704721FA02F3D040C2F120029140084306
:1072C0001946704710B5141E73F1000408DA401C0B
:1072D00041F1000192185B411A4301D120F00100F5
:1072E00010BD2DE9F04D92469B4611B1B1FA81F2E5
:1072F00002E0B0FA80F22032904600F053F80446E3
:107300000F4640EA0A0041EA0B0153465A46084339
:1073100013D0114653EA010019D0C8F1400250467B
:10732000FFF7C0FF05460E4650465946424600F05C
:1073300039F8084305D0012004E020463946BDE86D
:10734000F08D0020054346EAE0762C4337430A9847
:107350006305E40AA0EB08000022FD0A44EA475452
:107360000A3002D500200146E9E7010510196941FC
:10737000DDE9084500196941BDE8F04DA2E70000CC
:10738000064C074D06E0E06840F0010394E8070072
:1073900098471034AC42F6D3FFF7ACFED0EF0008AC
:1073A000F0EF0008202A04DB203A00FA02F1002066
:1073B00070479140C2F1200320FA03F31943904033
:1073C000704721B1826842F00102826003E0826866
:1073D00022F001028260704721B1826842F480721B
:1073E000826003E0826822F480728260704700004D
:1073F00010B504461248844208D10121401500F01E
:1074000099FC0021601500F095FC17E00D488442BE
:1074100008D10121001500F08DFC0021201500F09D
:1074200089FC0BE00848844208D10121C80300F020
:1074300081FC00214FF4004000F07CFC10BD0000F6
:107440000024014000280140003C0140014600208A
:107450008A6802F004020AB1012000E000207047AF
:10746000014600208A6802F008020AB1012000E00B
:107470000020704730B502460020002350680F4CB2
:1074800020400D790C6844EA052420435060906840
:107490000B4C2040D1E902542C434D7944EA450479
:1074A00020439060D06A20F470000C7C641EE4B22B
:1074B000234340EA0350D06230BD0000FFFEF0FFDE
:1074C000FDF7F1FFF0B504460D4600200021092D1F
:1074D00011DDE068A5F10A0606EB4607072606FA65
:1074E00007F18843A5F10A0606EB460603FA06F102
:1074F0000843E0600CE0206905EB4507072606FA23
:1075000007F1884305EB450603FA06F108432061BD
:10751000072A0FDA606B561E06EB86071F2606FA4F
:1075200007F18843561E06EB860605FA06F1084366
:10753000606322E00D2A0FDA206BD61F06EB860768
:107540001F2606FA07F18843D61F06EB860605FAC2
:1075500006F10843206310E0E06AA2F10D0606EB95
:1075600086071F2606FA07F18843A2F10D0606EBEF
:10757000860605FA06F10843E062F0BD816841F035
:1075800008018160704721B1826842F4A0028260E4
:1075900003E0826822F4A00282607047816841F0B3
:1075A00004018160704700BFFEE721B1026842F02C
:1075B0000102026004E002684FF6FE731A400260A6
:1075C0007047000001684FF6FE7211400160002113
:1075D000016041608160C1604B49884208D14A49DD
:1075E0000839496841F00F01474A083A51608AE07A
:1075F00045491431884208D143490839496841F066
:10760000F001414A083A51607DE03F492831884203
:1076100008D13D490839496841F470613A4A083A4D
:10762000516070E038493C31884208D13649083908
:10763000496841F47041344A083A516063E0324984
:107640005031884208D130490839496841F47021E5
:107650002D4A083A516056E02B496431884208D1DE
:1076600029490839496841F47001274A083A5160AC
:1076700049E025497831884208D1234908394968C9
:1076800041F07061204A083A51603CE01F4988424D
:1076900006D1011F096841F00F01021F116032E09D
:1076A0001A491431884208D11849091F096841F064
:1076B000F001164A121F116025E014492831884252
:1076C00008D11249091F096841F470610F4A121F5D
:1076D000116018E00D493C31884208D10B49091F5F
:1076E000096841F47041094A121F11600BE0074913
:1076F0005031884207D10549091F096841F47021BA
:10770000024A121F1160704708000240080402403C
:1077100010B50022026847F6F0739A430C6A8B6832
:1077200023430C6923434C6923438C692343CC696D
:1077300023434C6A23438C6A23431A430260CB6879
:1077400043600B6883604B68C36010BD70470000E6
:1077500004200B49C96801F0010109B101200EE0C4
:107760000749C96801F0040109B1022007E0044992
:10777000C96801F0100109B1032000E0042070473E
:107780000020024000200449C96901F0020109B14A
:10779000012000E0002070470020024003480069FB
:1077A00040F080000149086170470000002002405D
:1077B00030B5054604244FF4302000F05BF8044651
:1077C000042C41D12148224988602248886008461B
:1077D000006940F0200008610846006940F0400060
:1077E00008614FF4302000F045F80446042C22D103
:1077F0001748006941F6DF710840154908610846DD
:10780000006940F0100008611DB100201249088095
:1078100002E0A520104908804FF4302000F02AF83B
:107820000446052C10D00A48006941F6EF71084063
:107830000749086108E0052C06D00548006941F6B3
:10784000DF71084002490861204630BD23016745C9
:1078500000200240AB89EFCD00F8FF1F024803492A
:107860004860034848607047230167450020024094
:10787000AB89EFCD00B502460423FFF769FF03464D
:1078800003E0FFF765FF0346521E012B01D1002ADA
:10789000F7D102B90523184600BD000008B5012143
:1078A00040F21D2000F036FA0121084600F032FABD
:1078B0000121042000F02EFA0121082000F02AFA0C
:1078C0000121102000F026FA0121202000F022FAE8
:1078D00001210D4800F0A8F88020ADF8000010202C
:1078E0008DF8030003208DF802006946074800F078
:1078F0000FF800208DF803002020ADF80000694645
:10790000024800F005F808BD000230000008014000
:107910002DE9F04102460025002600200023002426
:10792000002791F803C00CF00F0591F803C00CF08C
:10793000100CBCF1000F03D091F802C04CEA050511
:1079400091F800C0BCF1000F31D0146800202BE08A
:107950004FF0010C0CFA00F3B1F800C00CEA03067A
:107960009E4220D183004FF00F0C0CFA03F7BC436A
:1079700005FA03FC4CEA040491F803C0BCF1280F9B
:1079800006D14FF0010C0CFA00FCC2F814C00AE05A
:1079900091F803C0BCF1480F05D14FF0010C0CFA6F
:1079A00000FCC2F810C0401C0828D1D31460B1F804
:1079B00000C0BCF1FF0F34DD546800202EE000F160
:1079C000080C4FF0010808FA0CF3B1F800C00CEAFB
:1079D00003069E4221D183004FF00F0C0CFA03F7EF
:1079E000BC4305FA03FC4CEA040491F803C0BCF163
:1079F000280F05D100F1080C08FA0CF8C2F8148021
:107A000091F803C0BCF1480F07D100F1080C4FF00A
:107A1000010808FA0CF8C2F81080401C0828CED3E0
:107A20005460BDE8F0810000F0B50A460023002450
:107A30000021002500F00046B6F1004F02D11D4E96
:107A4000F16901E01B4E7168C0F3034583B200F495
:107A50004016B6F5401F08D121F07061154E7668CA
:107A600026F07066134F7E6012E000F48016B6F5C3
:107A7000801F06D1032606FA05F4A14341F0706188
:107A800006E0460D360103FA06F6B14341F0706197
:107A900022B1460D360103FA06F6314300F00046E6
:107AA000B6F1004F02D1034EF16101E0014E716069
:107AB000F0BD0000000001400146C86880B2704778
:107AC00002460020D3680B400BB1012000E00020EB
:107AD00070474161704701617047C16070470AB1EA
:107AE000016100E04161704706480068064908608E
:107AF0000448001D0068486002480830006888603B
:107B000070470000E8F7FF1F5021002000BFFEE78C
:107B100010B503F081F94FF480710F48FFF7DBFFD8
:107B200040210E48FFF7D7FF02210C48FFF7D3FF93
:107B30004FF400710848FFF7CCFF4FF47A7002F061
:107B400005F94FF400710448FFF7C5FF4FF4FA70D0
:107B500002F0FCF810BD0000000C014000080140DC
:107B600070B504464FF400511148FFF7B2FF03F01F
:107B7000E7F81048FFF7A0FF00F47F4040EA040553
:107B800029460C48FFF7A9FF4FF480710948FFF719
:107B9000A0FF02210848FFF79CFF02210648FFF7DB
:107BA0009AFF4FF480710348FFF795FF70BD000006
:107BB00000100140000C01400008014070B504466F
:107BC0004FF400511148FFF786FF03F0B9F8104851
:107BD000FFF772FF00F47F4040EA040529460C4895
:107BE000FFF77BFF4FF480710948FFF772FF022116
:107BF0000848FFF76EFF02210648FFF76CFF4FF4BD
:107C000080710348FFF767FF70BD0000001001405E
:107C1000000C01400008014000BFFEE7704710B5AE
:107C20004FF4A06000F03AF810BD000070B50021DC
:107C300000230F22C47804B3154C246804F4E064D4
:107C4000C4F5E064210AC1F10403CA40447804FA8F
:107C500003F184781440214309010E4C0678A155A4
:107C6000047804F01F050124AC4005786D11AD00C7
:107C700005F1E025C5F8004109E0047804F01F058E
:107C80000124AC40044D0678761145F8264070BDBD
:107C90000CED00E000E400E080E100E00249014377
:107CA000024A1160704700000000FA050CED00E088
:107CB000014908627047000000000E4201460020A2
:107CC000034A506820F44040084350607047000069
:107CD0000010024029B1064A52690243044B5A611E
:107CE00004E0034A52698243014B5A617047000025
:107CF0000010024029B1064AD2690243044BDA61FE
:107D000004E0034AD2698243014BDA617047000004
:107D10000010024029B1064A92690243044B9A615D
:107D200004E0034A92698243014B9A617047000064
:107D30000010024029B1064AD2680243044BDA60BF
:107D400004E0034AD2688243014BDA6070470000C6
:107D50000010024030B500210022002400232D4DE8
:107D60006D6805F00C0121B1042905D0082923D143
:107D700005E0294D056022E0284D05601FE0254DF6
:107D80006D6805F47012234D6D6805F4803402258A
:107D900005EB92421CB9224D554305600BE01D4D89
:107DA0006D6805F400351DB11B4D5543056002E0BB
:107DB0001A4D5543056002E0174D056000BF00BF36
:107DC000144D6D6805F0F0010909164D6B5C0568EE
:107DD000DD4045600F4D6D6805F4E061090A114D05
:107DE0006B5C4568DD4085600A4D6D6805F4605147
:107DF000C90A0C4D6B5C4568DD40C560054D6D687A
:107E000005F44041890B084D6B5CC568B5FBF3F583
:107E1000056130BD0010024000127A000024F40019
:107E200000093D000000002010000020014908600A
:107E3000704700003C044242704710B500F002F861
:107E400010BD00000CB50020019000903348006880
:107E500040F480303149086000BF3048006800F4C9
:107E6000003000900198401C0190009820B94FF616
:107E7000FF7101988842F0D12848006800F4003072
:107E800010B10120009001E000200090009801282E
:107E900043D12348006840F010002149086008469B
:107EA000006820F0030008600846006840F0020007
:107EB00008601A48406819494860084640684860A8
:107EC0000846406840F4806048600846406820F4F6
:107ED0007C1048600846406840F4F8104860084646
:107EE000006840F08070086000BF0C48006800F037
:107EF00000700028F9D00948406820F003000749C5
:107F000048600846406840F00200486000BF0348EF
:107F1000406800F00C000828F9D10CBD00100240A8
:107F200000200240042808D14FF0E021096941F007
:107F300004014FF0E022116107E04FF0E0210969F0
:107F400021F004014FF0E0221161704710B5124892
:107F5000006840F0010010490860084640680F4979
:107F600008400D494860084600680D4908400A4924
:107F700008600846006820F48020086008464068D1
:107F800020F4FE0048604FF41F008860FFF755FFA3
:107F900004480549086010BD001002400000FFF8C9
:107FA000FFFFF6FE0070000808ED00E0F0B50C469B
:107FB000154600220021068C4FF6FE773E400684CF
:107FC000028B018C4FF60C7632407E1C06EA0316BB
:107FD0002E433243104EB0420ED0104EB0420BD062
:107FE000B0F1804F08D00E4EB04205D00D4EB042D9
:107FF00002D00D4EB04206D14FF6FD76314044F02E
:108000000106314305E04FF6F576314044F00106B4
:10801000314302830184F0BD002C01400034014053
:108020000004004000080040000C0040F0B50C4681
:108030001546002200210026078C4FF6EF7C07EA48
:108040000C070784028B018C4FF6FF7707EA0416B2
:1080500040F6FF473A404FF6FF7707EA03373A43C7
:108060004FF6FF7707EA05273A43114FB8420ED083
:10807000104FB8420BD0B0F1804F08D00E4FB8422D
:1080800005D00E4FB84202D00D4FB84206D14FF680
:10809000DF77394046F01007394305E04FF65F7748
:1080A000394044F01007394302830184F0BD0000D9
:1080B000002C014000340140000400400008004052
:1080C000000C0040F0B50C461546002200210026A9
:1080D000078C4FF6FF6C07EA0C070784828B018C34
:1080E0004FF6FF7707EA04264FF60C773A404FF633
:1080F000FF7707EA03172F433A43114FB8420ED0D8
:10810000104FB8420BD0B0F1804F08D00E4FB8429C
:1081100005D00E4FB84202D00D4FB84206D14FF6EF
:10812000FF57394046F48077394305E04FF2FF5757
:10813000394044F48077394382830184F0BD0000E4
:10814000002C0140003401400004004000080040C1
:10815000000C0040F0B50C46154600220021002618
:10816000078C4EF6FF7C07EA0C070784828B018C94
:108170004FF6FF7707EA043640F6FF473A404FF6DE
:10818000FF7707EA05273A434FF6FF7707EA0337F9
:108190003A43114FB8420ED0104FB8420BD0B0F155
:1081A000804F08D00E4FB84205D00E4FB84202D0D3
:1081B0000D4FB84206D14DF6FF77394046F480574F
:1081C000394305E047F6FF57394044F480573943B7
:1081D00082830184F0BD0000002C01400034014086
:1081E0000004004000080040000C004010B5734837
:1081F00004780121880700F081FBF0B16F48007816
:10820000012816D16E480078032803D104206C4958
:1082100008700EE06A480078082803D109206849F0
:10822000087006E0664800780D2802D10E206449E7
:1082300008700221480700F01FFC0221480700F0E7
:108240005DFB002873D04FF0804000F054FB5D4987
:1082500008805A480078012869D1594800780E28CA
:1082600076D2DFE800F09D072C829D9D082D839D2E
:108270009D092E8400BF00BF53480068D8B95048FC
:108280000078012803D102204D4908700EE04C48C7
:108290000078062803D107204949087006E04848BD
:1082A00000780B2802D10C204549087000214FF0BE
:1082B000804000F0E1FB00204449088071E000BFED
:1082C00000BF4148006800284ED03E48008844F670
:1082D000206188422CDC3B480088B0F57A7F27DBA0
:1082E00037480078022803D10320354908700EE092
:1082F00033480078072803D108203149087006E088
:108300002F4800780C2802D10D202D4908702D48E7
:1083100001882E4802880088401C2C4B1880181DAC
:1083200020F812100221480700F0A6FB1CE039E0FB
:1083300023480078022803D10120214908700FE06A
:108340001F480078072804D106201D49087007E05F
:1083500026E01B4800780C2802D10B201849087031
:108360000221480700F088FB1BE000BF00BF164851
:10837000006820B10221480700F07EFB04E00021E4
:108380004FF0804000F078FB0E4801880F480288CB
:108390000088401C0D4B1880181D20F8121000E0BA
:1083A00000BF00BF00214FF0804000F06EFB0321B2
:1083B0004FF0804000F07EFA10BD00004A0000201F
:1083C000470000204000002000012142220200203E
:1083D00008B50121404800F091FA00287AD0012127
:1083E0003D4800F06AFA00213B4800F069FA00219C
:1083F000394800F04AFB39480088394909888842E1
:108400004ADD3648001D3649098830F811003249E6
:108410002C3108803248007800F00100D8B10121E9
:108420000420FFF777FC4FF48070ADF800001020B7
:108430008DF8030003208DF8020069462948FFF7F4
:1084400067FA4FF480712748FFF743FB0021264865
:1084500000F042FA16E0012140F60500FFF75AFC51
:108460004FF48070ADF8000018208DF80300032051
:108470008DF8020069461B48FFF74AFA01211A48A5
:1084800000F02AFA0121144800F01AFA1448008872
:10849000401C134908801DE001210420FFF73AFC2D
:1084A0004FF48070ADF8000010208DF80300032019
:1084B0008DF8020069460B48FFF72AFA4FF48071E5
:1084C0000848FFF706FB0021074800F005FA0020E6
:1084D0000649087008BD000000040040C01B0020D1
:1084E0004C00002000080140002C01404500002005
:1084F0007FB505460C4601210220FFF7FBFBADF8D6
:108500000450ADF800400020ADF80600ADF80200C0
:1085100069460E4800F0E8FA012211460B4800F0C7
:1085200055FA1D208DF80C0001208DF80D00032058
:108530008DF80E0001208DF80F0003A8FFF776FBE1
:108540000121024800F0BCF97FBD0000000400409A
:1085500010B50121984800F0D1F900287ED0012102
:10856000954800F0AAF995480078401CC0B293499C
:108570000870042873DB0020087091480068401CD4
:108580008F4908608F480078401CC0B28D49087040
:108590000A2805DB01208C490870002089490870F1
:1085A0008A480088401C80B288490880FA2825DB68
:1085B000002008800120864908708648007801283C
:1085C0000DD1C1038448FFF77BFAC0F10100C4B2AA
:1085D00022464FF400418048FFF781FA0EE07F48C1
:1085E0000078FF2805D14FF400417B48FFF773FA6C
:1085F00004E04FF400417848FFF76BFA78480088B0
:10860000401C80B276490880B0F5FA7F04DB002078
:10861000088001207349087073480088401C80B2AC
:1086200071490880B0F57A7F64DB00200880012062
:108630006E4908706E480078FF2808D06D480078B1
:10864000022804D06A480078401E694908706A48C8
:108650000078401CC0B26849087001E0ABE095E0CA
:10866000052810DB052008706448007801280AD02E
:1086700000205A4908704FF400415748FFF729FA83
:1086800001205E4908705E480078401CC0B25C4919
:108690000870052814DB0520087058480078032866
:1086A00003D05648007802280AD1022053490870A6
:1086B00000204A4908704FF400414748FFF709FA83
:1086C00046480078FF2837D04A48007898B94B4888
:1086D000007803280FD141480078401CC0B23F49C0
:1086E00008703C282DDBFF2008704FF400413A4809
:1086F000FFF7F1F925E041480078022808D1002071
:10870000364908704FF400413348FFF7E2F918E0AA
:108710003A480078012814D130480078401CC0B293
:108720002E4908703C280CDBFF2008704FF40041F4
:108730002948FFF7D0F904E04FF400412648FFF73D
:10874000CAF930480078401CC0B22E49087023286E
:1087500008DB0020087000F065FE2B49088001202E
:108760002A4908702A480078401CC0B2284908707D
:10877000062801DB0620087026480078401CC0B29D
:1087800024490870062801DB06200870224800787A
:10879000FF2810D020480078401CC0B21E49087045
:1087A000042808DB08460078142801DBFF20087045
:1087B00001201A49087010BD000800403800002050
:1087C0003C0000203000002028000020360000205F
:1087D0002E00002018000020000801406200002048
:1087E000320000202B000020340000202C0000204C
:1087F000D1000020CF00002061000020320C0020BA
:10880000600000209C0000209E0000209D000020B1
:10881000DB000020DC0000201A00002019000020EE
:108820007FB505460C4601210420FFF763FAADF839
:108830000850ADF804400020ADF80A00ADF806007D
:1088400001A90E4800F050F9012211460B4800F032
:10885000BDF81E208DF8000002208DF801000320D5
:108860008DF8020001208DF803006846FFF7DEF95D
:108870000121024800F024F87FBD000000080040FC
:108880000246074B10681B68181A01EB4103C3EB43
:10889000C113B0EBC30F01D9012070470020FCE7E2
:1088A0003C00002001460248006808600120704733
:1088B0003C000020CA4302827047CA4302827047CC
:1088C00021B1028842F00102028004E002884FF6E2
:1088D000FE731A400280704731B1B0F8442042F470
:1088E0000042A0F8442005E0B0F84420C2F30E0294
:1088F000A0F8442070470146888E704730B5024684
:10890000002000230024158A05EA0103958905EA61
:10891000010413B10CB1012000E0002030BD0000C3
:1089200070B505460C46244885420ED02348854242
:108930000BD0B5F1804F08D02148854205D02148A1
:10894000854202D02048854200D100E000BF208847
:1089500050B92389A28861882846FFF727FBE18860
:10896000284600F094F825E0208804280AD12389BD
:10897000A28861882846FFF759FBE188284600F065
:108980008FF817E0208808280AD12389A2886188F7
:108990002846FFF797FBE188284600F08EF809E0AB
:1089A0002389A28861882846FFF7D4FBE1882846FE
:1089B00000F08CF870BD0000002C01400034014034
:1089C0000004004000080040000C00401AB18389F8
:1089D0000B43838102E083898B43838170470000CE
:1089E00070B5002400220023058C4FF6FE7635403A
:1089F0000584028C8388048B4FF68F752C40B51E3E
:108A00002C400D882C43751E2A400D892A434D8821
:108A10002A43144DA8420BD0134DA84208D0134D41
:108A2000A84205D0124DA84202D0124DA84213D13F
:108A30004FF6F7752A404D892A434FF6FB752A40B9
:108A40008D882A434FF6FF652B404FF6FF552B408C
:108A50008D892B43CD892B4383800483CD888586E4
:108A6000028470BD002C01400034014000400140F0
:108A700000440140004801400A460021018C4FF6A5
:108A8000FD73194011430184704781847047028B44
:108A90004FF6F3731A400283028B0A430283704736
:108AA000028B4FF2FF331A400283028B4FF6FF73A3
:108AB00003EA01231A4302837047828B4FF6F37354
:108AC0001A408283828B0A4382837047828B4FF2E3
:108AD000FF331A408283828B4FF6FF7303EA012330
:108AE0001A43828370470000002202881D4B98427F
:108AF0000ED01D4B98420BD0B0F1804F08D01B4BCD
:108B0000984205D01A4B984202D01A4B984204D191
:108B10004FF68F731A404B881A43174B984207D071
:108B2000164B984204D04FF6FF431A40CB881A43A5
:108B300002808B8883850B8803850A4B98420BD073
:108B4000094B984208D00E4B984205D00D4B9842E5
:108B500002D00D4B984201D10B7A03860123838208
:108B600070470000002C0140003401400004004028
:108B700000080040000C00400010004000140040BD
:108B800000400140004401400048014030B589B038
:108B900000BF00BF012140F60500FFF7BBF84FF40E
:108BA0008070ADF8200018208DF8230003208DF888
:108BB000220008A92F48FEF7ABFE2F48006849F2B3
:108BC0007041B0FBF1F0401E84B2601E4FF425717D
:108BD00048434FF47A71B0FBF1F085B20020ADF854
:108BE0001400ADF81600ADF81840ADF81A008DF875
:108BF0001C0005A92148FFF777FF7020ADF804009D
:108C00000120ADF806000420ADF80800ADF80A50C8
:108C10000220ADF80C000020ADF80E00ADF81000F9
:108C20004FF48070ADF8120001A91448FFF7D8FE88
:108C300001211248FFF744FE00211048FFF74CFEC7
:108C400001210420FFF766F84FF48070ADF8200092
:108C500010208DF8230003208DF8220008A9054874
:108C6000FEF756FE4FF480710248FEF732FF09B05E
:108C700030BD00000008014088000020002C0140A9
:108C800000B587B001210846FFF734F84FF6FF70B2
:108C9000ADF810006B20ADF80C000020ADF812000C
:108CA000ADF80E0003A94FF08040FFF71DFF002034
:108CB000ADF800000220ADF802000120ADF804007C
:108CC0000020ADF806000320ADF8080069464FF01B
:108CD0008040FFF725FE01218807FFF7F1FD1C20EA
:108CE0008DF8180001208DF8190003208DF81A0066
:108CF00001208DF81B0006A8FEF798FF0122032132
:108D00009007FFF763FE07B000BD0000124800881F
:108D1000124908701048001D008808700846007845
:108D200008700F480078012810D00E4800687F288E
:108D300009D2084601780B4802680068401C094BBC
:108D40001860094881540020084908704FF6F770F0
:108D500001490880704700000038014024000020CD
:108D6000190000201C000020000100201A00002033
:108D700021B1828942F40052828104E082894DF659
:108D8000FF731A408281704702460020B1F5007FD0
:108D900000D100BF13880B400BB1012000E0002080
:108DA0007047F0B50346002400260025002040F659
:108DB0006A17B94200D100BF1846C1F3421401F04E
:108DC0001F06012707FA06F5012C01D10C3004E03B
:108DD000022C01D1103000E014301AB107682F4383
:108DE000076002E00768AF430760F0BD2DE9F04778
:108DF00086B005460E460024A24600BFA1460027C5
:108E0000B08900B100BF2F462C8A4CF6FF70044099
:108E1000F08804432C82AC894EF6F3100440B088ED
:108E200031890843718908430443AC81AC8A4FF609
:108E3000FF400440B0890443AC8201A8FEF78AFFDA
:108E40001F48874202D1DDF810A001E0DDF80CA038
:108E5000A88900F4004040B10AEBCA0000EB0A10F8
:108E600031684900B0FBF1F807E00AEBCA0000EBFB
:108E70000A1031688900B0FBF1F86420B8FBF0F00B
:108E800004012009642101FB1089A88900F4004035
:108E900040B1322000EBC900B0FBF1F000F0070058
:108EA000044308E0322000EB09106421B0FBF1F02C
:108EB00000F00F0004432C8106B0BDE8F0870000ED
:108EC00000380140C1F308028280704700BFFEE70E
:108ED0000FB4084B10B504A902AA039800F01CF8BF
:108EE000044602A9002000F0B8F9204610BC5DF845
:108EF00014FB00005B92000802E008C8121F08C1C2
:108F0000002AFAD170477047002001E001C1121F0A
:108F1000002AFBD1704700002DE9FF4F8BB0884637
:108F20000546002606E025280BD0DDE90D12904706
:108F30006D1C761C28780028F5D10FB03046BDE8AE
:108F4000F08F0024A146A2460122AE4900E004436E
:108F500015F8013F203B02FA03F00842F7D12878C8
:108F60002A2810D06FF02F022878A0F130010929AB
:108F700015D809EB890102EB410144F0020400EB32
:108F800001096D1CF0E758F8041B5FEA010903D5DD
:108F900044F40054C9F1000944F002046D1C28781F
:108FA0002E2817D115F8010F44F004042A280ED0FA
:108FB0006FF02F022878A0F1300109290AD80AEBB6
:108FC0008A0102EB410100EB010A6D1CF2E758F83F
:108FD00004AB6D1C28786C280FD006DC4C2817D009
:108FE00068280DD06A2814D104E0742810D07A289B
:108FF0000FD10DE044F400140AE044F4801401E0C1
:1090000044F440146978814202D104F580146D1C47
:109010006D1C2878692865D006DC00288DD063286F
:1090200027D0642806D15DE06E2808D073282AD0A6
:10903000752877D0DDE90D129047761CE0E0C4F387
:109040000250022809D003280DD0D8F800100428B7
:109050000DD00E6008F10408D2E0D8F80010F21725
:10906000C1E90062F6E7D8F800100E80F2E70E7052
:10907000F0E718F8041B8DF8001000208DF80100AF
:10908000EB46012003E058F804BB4FF0FF306107C6
:109090004FF0000701D40AE07F1C57450DDA8742E4
:1090A000FADB1BF807100029F6D106E07F1C874287
:1090B000FCDB1BF807100029F8D1DDE90D23A9EB33
:1090C00007008146214600F0B1F83044C61904E09B
:1090D000DDE90D121BF8010B90477F1EF8D22146E7
:1090E000484688E058F8040BC4F302514FF00A0BCD
:1090F000032900D100B2042900D140B2002802DACD
:1091000040422D2102E0210505D52B218DF82410A8
:10911000012104E006E0E10710D02021F6E708AFC6
:10912000089113E058F8040BC4F302514FF00A0BF6
:10913000032900D180B2042900D1C0B20021EEE79A
:109140005946FEF799F8303107F8011D0028F7D18C
:10915000ADEB070000F1200B600702D524F480344A
:1091600001E04FF0010ADA4502DDAAEB0B0000E056
:109170000020824600EB0B0108980144A9EB010096
:109180000A90E00306D4DDE90D2321460A9800F099
:109190004DF806444FF0000908E009A911F809004C
:1091A000DDE90D12904709F10109761C08998945FE
:1091B000F3DBE0030CD5DDE90D2321460A9800F02E
:1091C00035F8064404E0DDE90D1230209047761CA6
:1091D000BAF10001AAF1010AF5DC05E0DDE90D12A2
:1091E00017F8010B9047761CBBF10001ABF1010BA6
:1091F000F4DC0A982146DDE90D2300F005F8064469
:109200006D1C97E6092801002DE9F0410446002570
:109210001E461746880404D405E039462020B0478E
:109220006D1C641EF9D52846BDE8F0812DE9F0419A
:10923000044600251E469046C80301D5302700E0AD
:109240002027880404D505E041463846B0476D1C08
:10925000641EF9D52846BDE8F0810A68531C0B60EE
:109260001070704700B585B04FF48040FEF726FDC2
:109270001C48FEF7BDF80020009001208DF8040086
:109280008DF805004FF4602002900020039001202B
:109290008DF8100069461348FEF7ECF80723012209
:1092A00005211048FEF70EF901210E48FEF794F84B
:1092B00001210C48FEF785F80A48FEF75FF900BF68
:1092C0000848FEF7CDF80028FAD10648FEF766F9FF
:1092D00000BF0448FEF7BAF80028FAD100F07EFD7E
:1092E00005B000BD00240140002205E011F8013B5B
:1092F00000F8013B531CDAB20C2AF7DB7047000080
:1093000010B5482000F0FCFC01214FF0C050FEF7E2
:10931000F1FC0120FEF7CCFC0120FEF787FDFEF7F3
:109320007EFCFEF7BBFAFEF7F3FBE220FEF718FC2B
:10933000E020FEF715FCAF20FEF712FCA220FEF79E
:109340000FFCA020FEF70CFCC020FEF709FCAC20AF
:10935000FEF706FCA620FEF703FCA420FEF700FCA7
:109360002C20FEF7FDFB2E20FEF7FAFB2F20FEF748
:10937000F7FB2520FEF7F4FB8120FEF7F1FB3F20F1
:10938000FEF7EEFBD520FEF7EBFB0020FEF7E8FB37
:10939000D220FEF7E5FB0020FEF7E2FB4020FEF7BF
:1093A000DFFBB020FEF7DCFB1020FEF7D9FB00202E
:1093B000FEF7D6FBAF20FEF7D3FB00F051FEFFF720
:1093C00051FF01211248FEF7DEF801211148FEF796
:1093D000ECF8114800681149B0FBF1F0401E84B26E
:1093E00021460120FFF784F80B4800680C49B0FBC8
:1093F000F1F0401E84B22146FA20FFF711FAFFF780
:109400003FFCFFF7C3FB4FF4164003F061FB10BDB8
:109410000024014008000240880000202A2C0A0095
:1094200040420F0030B50023114802880488002113
:1094300015E00F4830F81100904202D90C4830F87E
:1094400011200B4830F81100A04202D2084830F831
:109450001140074830F811000344481CC1B20829E4
:10946000E7DB981A001B0625B0FBF5F080B230BD93
:109470000002002030B50246002309E012F8014B3B
:1094800011F8015BAC4201D0012030BD581CC3B2C1
:109490000C2BF3DB0020F8E70146002206E011F870
:1094A000013B0BB101207047501CC2B20C2AF6DB05
:1094B0000020F8E710B50448007820B100200249E8
:1094C000087001F0E7F910BD9D0000202DE9F04182
:1094D0000446002514B90020BDE8F0813E493F480C
:1094E000FFF7C8FFC0B13C48FFF7D6FF08B1002026
:1094F000F2E700203A4908703A48007818B1394834
:109500000078012802D102203649087036480078D8
:10951000012801D00020DFE70020314908703148E0
:10952000007818B12F480078012802D102202D4977
:1095300008702948007B0F280DD02748007B102891
:1095400009D02548007B042805D02348007B01284A
:1095500001D00020C0E7601E1F49095CA01E1E4A02
:10956000105C41EA0027A01E81B2104600F0A6FB65
:109570000646B74201D00020AEE71748007B04281A
:1095800003D100F037F8054606E01348007B1028A9
:1095900002D100F0EDFA05467DB12946134800F0EE
:1095A0008DFB064632122846691CCDB20F490A547B
:1095B0002846691CCDB20D490E5407490748FFF7EC
:1095C00059FF38B90320074908700020084908707E
:1095D0000549087028467FE700010020502100203F
:1095E00061000020320C00201800002080010020C3
:1095F0006000002070B51548807B1449497B40EA23
:109600000120C5B21148007C1049C97B40EA012005
:10961000C6B2642D01D0002070BD0D490D48FFF782
:1096200063FE0C4C0C34042004F8010B7006000E91
:1096300004F8010B642D05D1002004F8010B06206D
:1096400004F8010B0348201AC0B2E5E7000100202E
:10965000502100208001002010B5FE48007813281A
:1096600075D2DFE800F074FEFDFC0A1FFBFAF96119
:1096700075F8F7F6CCE0F5F4F3000520F54908702D
:109680000021084603F0CEFA28B90020F2490870FC
:10969000F249487402E00120EF490870F048FFF7F2
:1096A00001F918E20121EE48FFF7EAF800283AD064
:1096B000E948007888B90620E64908700020E949A1
:1096C0000870E648C07B012803D13220E649887043
:1096D00026E00A20E449887022E00120DD49087074
:1096E0000220E24908700021E14802F04DF81E20F6
:1096F00000F000FB00F09EFBD948FFF7D3F8D748F5
:10970000C07B012806D15F20DA4908803220DA497F
:10971000088005E02320D74908800A20D649088020
:10972000CF48FFF7BFF8D6E10A20CA4908700121E7
:10973000002003F077FA18B90020C749087002E04A
:109740000120C5490870C648FFF7ACF8C3E1C1E184
:109750000121C348FFF794F800284FD0BE48007895
:1097600078BBC1488178BD481630BE4A1278815412
:109770000B20B8490870BC488078B8498874BA484A
:109780008078C874B7480078401CB6490870B6485D
:109790008078401CB449887008468078401CB549E0
:1097A0000880B1488078B4490880AC48C07B012863
:1097B00008D1B048008863281DDD6320AD490880CA
:1097C00019E007E0AB480088262814DD2620A949C7
:1097D000088010E006209F4908700020A149087009
:1097E0009E48C07B012803D132209F49887002E047
:1097F0000A209D4988709A48FFF754F86BE10F20C2
:109800009449087001219748007803F00BFA18B9C1
:1098100000209149087002E001208F4908709048AB
:10982000FFF740F857E101218D48FFF729F800289C
:1098300072D08948007800287FD18B48807887498A
:10984000C87489488178854816300BE0A6E08BE023
:109850007AE0E5E0E3E0E1E0DFE0DDE0DBE0D9E075
:10986000D7E0D5E07F4A127881547E480078401CCA
:109870007C4908700846007818280ADB10207549D2
:10988000087000217D4801F07FFF7548FFF70AF856
:1098900024E07248C07B012810D173488078632887
:1098A00003DB11206B49087018E00B206949087030
:1098B0006D488078401C6C4988700FE06A48807859
:1098C000262803DB11206349087007E00B2061495B
:1098D000087065488078401C634988706048FEF7CE
:1098E000E1FF61488078401C624908805E488078CA
:1098F000614908805948C07B01280FD15D48008824
:10990000632802DD63205B4908805748807863281C
:1099100019DD63205449887015E00EE05548008831
:10992000262802DD2620534908804F4880782628C3
:1099300009DD26204C49887005E00B204549087058
:109940004748FEF7AFFFC6E002214548FEF798FF03
:1099500048B111203F4908704148FEF7A3FF00219C
:10996000474801F011FFB6E078213D48FEF788FF37
:1099700098B100204349087036490870FF203749E4
:10998000C87488740120487400F054FA01203749E3
:10999000087000213A4801F0F7FE9CE003213048AE
:1099A000FEF76EFF18B30020364908702949087089
:1099B0002A480078032823D12848407CC0B90020D9
:1099C000314908702548007D2449C97B884207D168
:1099D00000202649087000212C4801F0D5FE16E031
:1099E0000120224908700021254801F0CDFE0EE03B
:1099F00001201E4908700021214801F0C5FE06E043
:109A000000201A4908700021204801F0BDFE62E0E4
:109A100000BF00BF00BF00BF00BF00BF00BF00BF4E
:109A200078210F48FEF72CFF90B3002009490870F9
:109A30001449087000F0FEF908480078032841D165
:109A40000648407CA8BB0548007D0449C97B884284
:109A500027D11EE04700002058000020320C0020D3
:109A6000500000205400002022020020CF000020DF
:109A7000B5B700086400002066000020F5BD0008AE
:109A8000F1BE00084A0000206A00002089B30008E7
:109A90001FE00020114908700021114801F074FEF8
:109AA00017E001200D49087000210E4801F06CFEFE
:109AB0000FE0FFE70120094908700021094801F083
:109AC00063FE06E00020054908700021044801F00B
:109AD0005BFE00E000BF00BF10BD0000CF00002013
:109AE00089B30008F1BE000870B51F48C07B50B9AB
:109AF0001D488089A0F5A07000EB8000092190FB33
:109B0000F1F085B201E0184885890A2095FBF0F054
:109B100085B21548407CD0B9134880884FF6FF7154
:109B2000884214D0002407E00F481630005DA84298
:109B300000DB06E0601CC4B20B48407D401EA04222
:109B4000F2DC00BF182C00DB17240848047007481B
:109B50000078182802DB17200449087003480078B1
:109B600000F03CFA70BD0000320C002070000020B4
:109B70002DE9F0414648807B4549497B40EA012672
:109B80004348007C4249C97B40EA0120C7B2C82E45
:109B900004DBD02E02DCF019CF2802DD0020BDE866
:109BA000F0813B4C1234002555E07019C838072865
:109BB0004ED2DFE800F0040C141C24384500607815
:109BC000217840EA012033498880A41C40E0607875
:109BD000217840EA01202F49C880A41C38E0607831
:109BE000217840EA01202B490881A41C30E06078EC
:109BF000217840EA012027494881A41C28E06078A8
:109C0000217840EA012023498873A41C0846807B00
:109C1000012803D10846C088888103E01D480089D7
:109C20001C49888114E06078217840EA01201949B4
:109C3000C8730846C07B184981F80605A41C07E0D4
:109C40006078217840EA012012490874A41C00BF02
:109C500000BF681CC5B2BD42A7DB10491048FFF722
:109C600043FB01220E490C3109480C3000F01AF870
:109C700002220B490D31104600F014F80222084967
:109C80000D3103480D3000F00DF80F2087E700007C
:109C900000010020320C0020220200205021002070
:109CA0008001002010B50346002003E01C5C0C542A
:109CB000441CE0B29042F9DB10BD000070B50246D2
:109CC0000C46FF25FF2309E012F8010B80EA05018D
:109CD0000648405C80EA03050548435C2000A4F187
:109CE0000106B4B2F0D143EA052070BD2ECE0008C3
:109CF0002ECF00080149087070470000D1000020F5
:109D000010B504464FF0E020006920F004004FF049
:109D1000E02108616FF00400FEF704F9E11704EB9D
:109D20005171C1F3C701074A11701046007800EB6A
:109D30004001C1EBC0104FF6FF7101EAC0000249BB
:109D4000088010BD1400002016000020002105E04E
:109D5000642200BF521E002AFCD1491C8142F7D95F
:109D6000704700000146114A12784A434FF0E02341
:109D70005A6100229A611A46126942F001021A6180
:109D800000BF4FF0E022106900F001021AB100F4A8
:109D90008032002AF5D04FF0E022126922F0010251
:109DA0004FF0E0231A6100229A61704714000020EE
:109DB00000200021084A00BF0BE0002004E000233F
:109DC00002F8013B431CD8B25F28F8DD01F108031B
:109DD000D9B24029F1DB70475C21002000B58BB07F
:109DE00001210846FDF776FF0F48FDF7EBFB0F4812
:109DF00000900F480190002002900820039000205E
:109E0000049080200590400006908000079020205C
:109E100008900002099000200A9069460248FDF768
:109E200077FC0BB000BD0000080002404C2401404C
:109E30000002002010B5082200210A4801F098FA1B
:109E400000240BE004EB84014FF6FF7202EA0120CC
:109E50000822044900F030F8601C84B2202CF1DBA9
:109E600010BD00000E210020F8B504460D46164630
:109E700000BF00BF0E4800780628FADB2B460222FE
:109E80002146A020009600F00DF9012806D10948CE
:109E9000007840F001000749087005E005480078A7
:109EA00020F0010003490870002001490870F8BD46
:109EB000DC00002059000020F8B504460D46164687
:109EC00000BF00BF0E4800780628FADB2B460222AE
:109ED0002146A020009600F0D7F9012806D10948B4
:109EE000007840F001000749087005E00548007857
:109EF00020F0010003490870002001490870F8BDF6
:109F0000DC0000205900002010B50648007838B168
:109F10000020044908700448407C08B900F008FAA1
:109F200010BD00002C000020320C002010B50848A5
:109F3000007860B100200649087002F0E9F90221BA
:109F40000448FEF79DFC10B100200349087010BDC5
:109F50002B0000205C0000201800002010B500211C
:109F6000084602F09DFA90B90A4800880A49A1F80B
:109F70004E050021084880F85015B0F84E250549D7
:109F8000091D00F2525002F0FFFC002010BD01201C
:109F9000FCE700002A070020320C002010B5012148
:109FA000002002F07DFA98B90A4800880A49A1F811
:109FB0006E0A08488178084880F8701AB0F86E2A4E
:109FC0000449091D00F6722002F0DEFC002010BDDD
:109FD0000120FCE72A070020320C002010B50446BF
:109FE0000121204602F05CFA80B90948008809493D
:109FF000C88507488178074880F83010C28D044929
:10A00000091D323002F0C0FC002010BD0120FCE729
:10A010002A070020320C0020002001E0411CC8B2B9
:10A020000828FBDB7047000008B501210420FDF77C
:10A0300071FE4FF4C050ADF8000014208DF80300FD
:10A0400003208DF8020069460448FDF761FC4FF4D7
:10A05000C0510248FDF73FFD08BD00000008014067
:10A0600010B5FFF7E1FF0E48006820F470400C497E
:10A0700008600846006840F44050086008460068E0
:10A0800020F4702008600846006840F44030086002
:10A09000C81403490C3108604000086010BD00007E
:10A0A000040801402DE9F84F06460C46154698462F
:10A0B000DDF828904FF0040A00BFCDF80090474625
:10A0C00006F0010060BB00F0A3F8FFF7A5FF3046E3
:10A0D00002F0E8FB10B100F0B7F847E0022D0ED116
:10A0E000C4F3072002F0DEFB10B100F0ADF83DE054
:10A0F000E0B202F0D7FB88B100F0A6F836E0012DFF
:10A1000006D1E0B202F0CEFB40B100F09DF82DE0A8
:10A1100025B900F099F80020BDE8F88F00F094F818
:10A12000FFF77AFF00F074F846F0010002F0BAFB86
:10A13000C8B900BF9DF80000401EC0B2009002F0F8
:10A14000FDFA07F8010B9DF8000010B102F074FB56
:10A1500001E002F03FFB9DF800000028EAD100F08A
:10A1600073F80020D8E700F06FF800BFAAF10100F3
:10A17000C0B25FEA000AA0D10120CDE710B500F01F
:10A1800047F80520FFF7EEFD4FF400601F49086017
:10A190000520FFF7E7FD1D481038006820F4702007
:10A1A0001A49103908600846006840F440300860D9
:10A1B0000520FFF7D7FD4FF480501449091F0860B0
:10A1C0000520FFF7CFFD002410E04FF400600F4999
:10A1D000091F08600520FFF7C5FD4FF400600B491B
:10A1E00008600520FFF7BEFD601CC4B2092CECDB43
:10A1F0000520FFF7B7FD00F00BF80520FFF7B2FDD3
:10A2000000F022F80520FFF7ADFD10BD1408014055
:10A2100010B50C48006820F470200A490860084610
:10A22000006840F440300860881406490C3108602A
:10A2300040100860FFF7F0FE4FF4805001491031E4
:10A24000086010BD0408014010B50E48006820F4F5
:10A2500070200C4908600846006840F440300860EF
:10A26000C814084910310860400008604010091FF8
:10A270000860FFF7D1FE4FF4805002490C310860AE
:10A2800010BD0000040801402DE9F05F81460C4636
:10A2900015461E46DDF828A04FF0040B00BFB0465F
:10A2A0005746FFF7B5FF484602F0FCFA10B1FFF73A
:10A2B000CBFF34E0022D0ED1C4F3072002F0F2FAF6
:10A2C00010B1FFF7C1FF2AE0E0B202F0EBFA88B16B
:10A2D000FFF7BAFF23E0012D06D1E0B202F0E2FA67
:10A2E00040B1FFF7B1FF1AE025B9FFF7ADFF00203D
:10A2F000BDE8F09F00BFFFF78FFE1FB9FFF7A4FF77
:10A300000020F5E718F8010B02F0CCFA00B102E0EA
:10A31000781EC7B2EFE700BFFFF796FF00BFABF1B3
:10A320000100C0B25FEA000BB9D10120E0E70000F4
:10A3300070B5BE488089BE490988884209D1BB48AA
:10A34000007CBC490978884203D1BB4800780728C3
:10A350004FD10020B9490870B9490870B948007850
:10A36000052813D0B748007806280FD0B5480078E4
:10A3700007280BD0B3480078082807D0B1480078E8
:10A38000092803D0AF4800780A2832D1AA480078BB
:10A39000072805D10020A8490870AA49087028E0BC
:10A3A000A2488089A249098888420BD09F4800783A
:10A3B000032802D10420A34908709C4880899C4945
:10A3C000088016E09948007C9A490978884210D0A4
:10A3D0009648007C974908709448007C18B904207E
:10A3E0009849087005E007209649087000209649B2
:10A3F0000870944800780B287ED2DFE800F0067DD4
:10A4000010171E2C538AAEB5FB0002208D49087030
:10A41000FFF7A4FD10B903208A49087004E1FFF793
:10A420009DFD10B9032087490870FDE0FFF7B6FDD8
:10A4300010B9042083490870F6E0FFF755FB48B9CE
:10A440007A48007C18B905207E49087002E0072090
:10A450007C490870E8E079480078012821D04FF461
:10A46000A4627A497A48FCF75DFE012073490870BE
:10A470000020784908807848007800F0080038B952
:10A48000012076490880012174482C38FEF718FA1B
:10A4900006206C4908707248FEF704FA00207149E2
:10A4A0000870C1E002216E48FEF7EAF910B96D4864
:10A4B000007868BB61480078012829D06848FEF719
:10A4C000F1F94FF4A46259492E316148FCF72AFE94
:10A4D00001205A49087000205E4908805E480078D3
:10A4E00000F0080038B901205C49088001215B4870
:10A4F0002C38FEF7E5F900E095E05A480078401C5A
:10A50000C0B258490870022802DB08204D49087083
:10A510008AE04A48007801281ED04FF4A4625249CC
:10A520004B48FCF7FFFD01204449087000204949D1
:10A5300008804948007800F0080038B901204749F0
:10A540000880012145482C38FEF7BAF90A203D4918
:10A5500008704648FEF7A6F966E04548FEF7A2F9FE
:10A560000920384908705FE04248007810B94FF47C
:10A57000967500E03C2529463D48FEF781F9B8B3C1
:10A5800001203C4908703A48FEF78CF927480078CA
:10A59000012813D12548407801280FD1234840884D
:10A5A00035490988884206DD2048408832490988B3
:10A5B000401A84B204E01D48448801E01B488488A6
:10A5C0001A4880896430A04204DB184880896438C6
:10A5D000A0420DDD1848007850B919480078401C99
:10A5E000C0B217490870032802DC0520154908701D
:10A5F0001AE0FFE74FF4E1611C48FEF741F988B12A
:10A600001A48FEF74FF910480078401CC0B20E49B6
:10A610000870032803DB0320087000BF02E0072056
:10A620000849087000BF00BF00BF70BD320C002099
:10A63000800000208200002048000020450000200B
:10A640006A0000204A00002083000020A01600209D
:10A65000C01B00204C000020590000202C040040AA
:10A660007C00002084000020801100207800002061
:10A6700074000020440000205600002010B521483E
:10A68000007848B920480078022805D101201D49EA
:10A6900008701E48FEF706F91D48007888B91D4865
:10A6A0000078FF2803D11E201A49087009E0032012
:10A6B000174908700021184801F066F80320FFF7D9
:10A6C00019FB1348007801281AD10F48407C28B99B
:10A6D0000D48C07B0C49097D884211D00D48007897
:10A6E000FF2803D11E200B49087009E00320084908
:10A6F00008700021084801F047F80320FFF7FAFA34
:10A7000010BD000018000020320C00205C0000206A
:10A71000CF000020CE00002085BE000810B500202C
:10A7200002F040F910BD000010B54F48007820B18C
:10A73000012820D0022874D156E04C480078032824
:10A740000AD10120484908700021494801F01CF84D
:10A750001E20FFF7CFFA0DE044480078012809D108
:10A760000420414908700021424801F00DF81E20E4
:10A77000FFF7C0FA75E03D480078032833D1FF2089
:10A780003A49C87488740020487501203A49087015
:10A790003A4908700220344908700120334948744E
:10A7A0000021374800F0F0FF3C20FFF7A3FAFFF745
:10A7B00041FB182200212D48163000F0D9FD2B480E
:10A7C000C07B012806D15F202E49088032202E4907
:10A7D000088005E023202B4908800A202A490880A8
:10A7E0002A48FEF75FF83CE023480078801F0C28D9
:10A7F0002CD2DFE800F00607082B2B1718192B2B9B
:10A800002B2000BF00BF01201849487411201A49AD
:10A810000870FF201549C87488741C48FEF742F878
:10A8200015E01DE000BF00BF112013490870174854
:10A83000FEF738F80BE0164800780C4948751220EE
:10A840000D4908701148FEF72DF800E000BF00BF69
:10A8500000210B4800F098FF1E20FFF74BFA00E0A4
:10A8600000BF00BF10BD0000CF000020320C002050
:10A87000F1BE0008ADBD0008470000204A000020DE
:10A88000B5B70008640000206600002050000020DA
:10A890005400002010B500207149087014E0714880
:10A8A0006F49097830F811006F490988884206DC41
:10A8B0006E486B490978405C6D49087008E068484B
:10A8C0000078401C66490870654800780628E6DB79
:10A8D00000BF6748007867490978884241D16448D9
:10A8E000007865490978884242D064480078401E63
:10A8F000C0B26249087000283AD161490870FF204F
:10A90000604908705A4800785B4908705E480978C9
:10A9100050F821005D490860084600685C4988429B
:10A9200018D05A4800685B49884213D057480068DD
:10A93000594988420ED0554800685849884209D084
:10A94000524800685649884204D05048006855492A
:10A95000884202D14D480068804700205249087063
:10A9600006E04348007843490870022043490870D4
:10A970004E480078FF2833D04C48007858BB4248F6
:10A980003D49097850F821004049086008460068B0
:10A990003F49884218D03D4800683E49884213D05C
:10A9A0003A4800683C4988420ED0384800683B4924
:10A9B000884209D0354800683949884204D0334874
:10A9C00000683849884202D1304800688047FF203B
:10A9D0003649087004E035480078401E3349087055
:10A9E00028480078FF2833D02648007858BBFF203D
:10A9F0002449087024482049097850F82100234947
:10AA00000860084600682249884218D01F4800683C
:10AA10002049884213D01D4800681F4988420ED043
:10AA20001A4800681D49884209D0184800681C4926
:10AA3000884204D0154800681A49884208D1134852
:10AA40000068804704E00F480078401E0D490870F8
:10AA50000948007810B100201349087010BD0000AB
:10AA6000CA0000201CCE00089E00002028CE00084E
:10AA7000CB000020C8000020C9000020CC0000202E
:10AA8000A3000020CD000020B0000020A80000207E
:10AA9000B1AA00081DA7000879AC00087DA600082F
:10AAA00029A70008D1AA000862000020CE000020DB
:10AAB000FF20044908700449087000200349087009
:10AAC00070470000CE000020CD000020A50000202F
:10AAD00010B560480078022866D15F4800781128D8
:10AAE00002D012284BD118E05C48007870B90620DB
:10AAF000594908705A48C07B012803D1322059496E
:10AB0000887006E00A205749887002E00B205249FD
:10AB100008705548FDF7C6FE45E000204E49087014
:10AB2000524908704E480078032820D14C48407C98
:10AB3000A8B94B48007D4A49C97B884207D100200B
:10AB40004449087000214A4800F01EFE16E001202A
:10AB5000404908700021474800F016FE0EE0012031
:10AB60003C4908700021434800F00EFE06E000203A
:10AB70003849087000213E4800F006FE13E0FF202F
:10AB80003749C87488740020384908700120344956
:10AB90004874FFF74FF901202E490870002135480D
:10ABA00000F0F2FD00BF54E02A480078012814D1DB
:10ABB0000020294908702A48407C002849D12848AB
:10ABC000C07B2749097D884243D100202149087074
:10ABD0000021274800F0D8FD3BE01E4800780328FC
:10ABE0002CD11F480078032820D11D48407CA8B9EB
:10ABF0001B48007D1A49C97B884207D100201549AE
:10AC0000087000211A4800F0BFFD22E00120114920
:10AC100008700021174800F0B7FD1AE001200D4927
:10AC200008700021134800F0AFFD12E00020094930
:10AC3000087000210E4800F0A7FD0AE005480078E2
:10AC4000042806D10020034908700021084800F0BC
:10AC50009BFD10BDCF0000204700002054000020C5
:10AC6000320C002022020020500000204A00002068
:10AC700089B30008F1BE000810B5012001F092FE72
:10AC800010BD2DE9F84F80468946154615F801ABF1
:10AC900015F8010B00900AF00707082F15D2DFE81E
:10ACA00007F00406080A0C0E101280240EE001249E
:10ACB0000CE002240AE0042408E0082406E0102442
:10ACC00004E0202402E0402400E000BF00BF4FF079
:10ACD000000B2AE0B9F1400F00DD2DE027460026E9
:10ACE0001CE008EB0600602800DD19E028783840F9
:10ACF00038B108EB0601C8B20122494602F06CF8EF
:10AD000006E008EB0601C8B20022494602F064F8EA
:10AD10007F100FB980276D1C701CC6B25645E0DB52
:10AD200000BF09F1010000F0FF095846411C01F085
:10AD3000FF0B00998842CDDB00BFBDE8F88F000013
:10AD400008B501210820FCF7E5FFFF20ADF8000061
:10AD500003208DF8020010208DF803006946094891
:10AD6000FCF7D6FD01210846FCF7D4FF0121064877
:10AD7000FCF75AFE1820ADF8000069460148FCF7C0
:10AD8000C7FD08BD000C0140000430000146012948
:10AD900004D0022911D005292DD11DE00822174B1E
:10ADA0001A700622164B1A700822164B1A705001A0
:10ADB000154A121A154B1A601EE010220F4B1A701A
:10ADC00008220F4B1A7010220E4B1A705001104AB5
:10ADD000121A0E4B1A600FE03022084B1A70102224
:10ADE000074B1A701822074B1A709001094A121A61
:10ADF000064B1A6000E000BF00BF7047E000002073
:10AE0000E8000020E90000205EDA0008E4000020ED
:10AE10002ED0000856DD000808B501211C20FCF7E3
:10AE200079FF4220ADF8000010208DF803000320C8
:10AE30008DF8020069461E48FCF76AFD40F2FF30BB
:10AE4000ADF8000010208DF8030003208DF80200FB
:10AE500069461848FCF75CFD4FF40050ADF800005F
:10AE600010208DF8030003208DF802006946124877
:10AE7000FCF74EFD01210846FCF74CFF01210F486D
:10AE8000FCF7D2FD4FF40040ADF8000003208DF830
:10AE9000020010208DF8030069460548FCF738FDD4
:10AEA0001820ADF8000069460248FCF731FD08BDE6
:10AEB00000080140000C0140001001400004300077
:10AEC0002DE9F04F04460D469046994600274FF075
:10AED000010B4D4507DD66B2444606F0FF086EB231
:10AEE0004D4606F0FF09A8EB040046B2A9EB0500A9
:10AEF0004FFA80FA29462046099A01F06DFF002E8C
:10AF000004DCA4EB080046B24FF0FF3B56451CDDC5
:10AF100018E0002F06DD681CC5B2AAEB0600384415
:10AF200047B202E007EB0A0047B204EB0B00C4B2E1
:10AF3000602C01DA402D00DB06E029462046099A04
:10AF400001F04AFF4445E4D11BE017E0002F07DD84
:10AF500004EB0B00C4B2A6EB0A00384447B201E090
:10AF6000B81947B2681CC5B2602C01DA402D00DB6D
:10AF700006E029462046099A01F02EFF4D45E5D10D
:10AF800000BFBDE8F08F00002DE9F0470746884676
:10AF9000924636480068364909780AFB01090025BF
:10AFA0005EE099F8006009F101093248007808284C
:10AFB00008DD4FF6FF7000EA062699F80000064308
:10AFC00009F101092B480078082823DC00241CE043
:10AFD00006F0800040B108EB0502D1B23A19D0B2B8
:10AFE000012201F0F9FE07E008EB0502D1B23A199F
:10AFF000D0B2002201F0F0FE4FF6FF7000EA4606E4
:10B00000602C00DD05E0601CC4B21A480078844260
:10B01000DEDB23E000241CE006F4004040B108EB36
:10B020000502D1B23A19D0B2012201F0D5FE07E0F3
:10B0300008EB0502D1B23A19D0B2002201F0CCFEE1
:10B040004FF6FF7000EA4606602C00DD05E0601C4C
:10B05000C4B2084800788442DEDB00BF681CC5B279
:10B060000548007885429CDBBDE8F087E4000020BD
:10B07000E0000020E8000020E900002070B505464F
:10B080000E46144615E00D4800782844602800DD7F
:10B0900012E00B4800783044402800DD0CE02278B4
:10B0A00031462846FFF770FF044800782844C5B2AF
:10B0B000641C20780028E6D100BF70BDE8000020A5
:10B0C000E90000202DE9F043804689461446002718
:10B0D000002630E02778641C4FF6FF7000EA07274F
:10B0E00020780743641C00251EE007F4004048B1A7
:10B0F00009EB0602D1B208EB0502D0B2012201F041
:10B100006BFE08E009EB0602D1B208EB0502D0B2F3
:10B11000002201F061FE4FF6FF7000EA4707602D44
:10B1200000DD05E0681CC5B2064800788542DCDB1E
:10B1300000BF701CC6B2044800788642CADBBDE876
:10B14000F0830000E8000020E900002000BFFEF7C7
:10B15000D7F8FCF717FB012806D0FCF77FFB01208E
:10B16000FCF726FBFCF71AFB01F046F90220FFF77B
:10B170000DFE6B480078FCF759F807460022694B32
:10B18000FBF7E2FF0546FCF75EF800F0FF0966A258
:10B1900012214846FFF772FF0220FFF7F7FD6049D2
:10B1A00009784906080E62A22621FFF767FF01F021
:10B1B00015FD4FF400416148FCF78BFC6048FDF73A
:10B1C00071FBFCF791FC01F05FFA00205D4908700B
:10B1D0005B48FDF767FB00BF5B480078012833D16F
:10B1E0005A480068102817D358480068802813D29E
:10B1F00057480078FF280FD054490878FEF766F9C1
:10B20000044634B10120534948702146524801F0A8
:10B21000B7FCFF204E4908704E4880884FF6FF71FA
:10B22000884206D14D48007840F008004B4908702C
:10B2300005E04A48007820F00800484908700020DE
:10B24000424908604049087002213D48FDF718FB5B
:10B250000028C1D03F48407CA8B93E48007D3D4908
:10B26000C97B884207D100203D49087000213D4834
:10B2700000F08AFA0EE001203949087000213A48AE
:10B2800000F082FA06E001203549087000213648B6
:10B2900000F07AFA00BFFEF70DF9FEF747FEFEF761
:10B2A00033FE32480078012801D1FEF7D5F926484F
:10B2B0000078012820D125480068102817D323489A
:10B2C0000068802813D222480078FF280FD01F4939
:10B2D0000878FEF7FBF8044634B101201D49487098
:10B2E00021461D4801F04CFCFF2019490870002040
:10B2F0001649086014490870164880884FF6FF7197
:10B30000884206D11548007840F0080013490870BB
:10B3100005E01248007820F0080010490870BAE7EC
:10B32000E800002000000C404152532D3100000085
:10B3300056455220312E362E3900000000080140BB
:10B340006C00002062000020190000201C0000207A
:10B350001A000020320C002080010020590000203B
:10B36000CF00002089B30008F1BE00084A00002089
:10B3700030B5034601E003F8011B1400A2F10105FA
:10B38000AAB2F8D130BD00002DE9F843002600270D
:10B39000D7480078401CC0B2D5490870022801DBAC
:10B3A00000200870D3480078032873D1D148C07BAF
:10B3B000C0B9D0488089A0F5A07000EB80000921B9
:10B3C00090FBF1F086B2CC48007800F0080090B90C
:10B3D000C8488088A0F5A07000EB800090FBF1F0D9
:10B3E00087B208E0C3488689C348007800F00800A7
:10B3F00008B9C04887880A2096FBF0F086B20A2078
:10B4000097FBF0F087B2BB48007C00286CD1052088
:10B41000FFF7BCFC3246B9A1B948FDF759FDB84A5F
:10B420000A211420FFF72AFEB348007800F0080034
:10B4300020B1B4A1B248FDF74BFD04E03A46AFA1FC
:10B44000AF48FDF745FDAE4A22211420FFF716FE56
:10B450000120FFF79BFCACA20F214420FFF70EFE5A
:10B46000A9A221214420FFF709FEA8A20221002061
:10B47000FFF704FEAA4991F8008008EBD871481044
:10B48000A8A23721FFF7FAFD9A48C07B012802D114
:10B49000A8A001E036E0A8A00246A8A19848FDF7C0
:10B4A00017FD974A14214820FFF7E8FD944A26210A
:10B4B0004820FFF7E3FD01201F234F22194600908B
:10B4C0001020FFF7FDFC012020234F221946009099
:10B4D0001020FFF7F5FC012021234F221946009090
:10B4E0001020FFF7EDFC00E10520FFF74FFC8C4931
:10B4F00091F8008008EBD871481091A21421FFF751
:10B50000BDFDF2E07B480078022823D10425FFF737
:10B510003DFC8DA229460020FFF7B0FD8E48007843
:10B520002844C5B2E81CC5B28CA229460020FFF70A
:10B53000A5FD894800782844C5B2E81CC5B2784901
:10B5400091F8008008EBD871481088A22946FFF7CF
:10B5500095FDCAE0674800780128C4D16548407865
:10B5600020B16548007800F0200068B10220FFF7A4
:10B570000DFC6B4991F8008008EBD87148107EA251
:10B580001821FFF77BFDB0E05A48C07B08BB594843
:10B590008089A0F5A07000EB8000092190FBF1F0FC
:10B5A00086B25448408877490988884206DD514868
:10B5B000408874490988401A84B201E04D484488A3
:10B5C000A4F5A07000EB8000092190FBF1F087B298
:10B5D00010E04848868940886A490988884206DD23
:10B5E0004448408867490988401A84B201E04148CC
:10B5F000448827460A2096FBF0F086B20A2097FB83
:10B60000F0F087B23B48007C002861D10520FFF7AD
:10B61000BDFB324639A13A48FDF75AFC384A0A21A7
:10B620001420FFF72BFD3A4634A13548FDF750FCB6
:10B63000334A22211420FFF721FD0120FFF7A6FB4A
:10B6400031A20F214420FFF719FD2FA22121442010
:10B65000FFF714FD2DA202210020FFF70FFD304956
:10B6600091F8008008EBD87148102EA23721FFF71F
:10B6700005FD2048C07B012801D12EA000E02EA0AE
:10B6800002462EA11E48FDF723FC1D4A1421482026
:10B69000FFF7F4FC1A4A26214820FFF7EFFC0120AF
:10B6A0001F234F22194600901020FFF709FC0120AC
:10B6B00020234F22194600901020FFF701FC0120A3
:10B6C00021234F22194600901020FFF7F9FB0CE0D0
:10B6D0000520FFF75BFB124991F8008008EBD87159
:10B6E000481017A21421FFF7C9FCBDE8F883000039
:10B6F000D3000020320C00205900002025336400C4
:10B70000F02000202D2D2D002E00000020202020D4
:10B71000536574706F696E74202020200000000053
:10B72000E80000202020202043757272656E74208E
:10B730002020200046000000430000002573000088
:10B74000204F464620000000506C656173652070F4
:10B750007265737300000000E900002020416464FA
:10B7600072657373696E672000000000202020203E
:10B770006B6579202020200020206F66666C696E42
:10B78000652020005600002070B504460D4644B1E7
:10B79000FEF70EFB15B12846A04700E0A04701F0D8
:10B7A0001DFA024800780249087070BDCF000020E1
:10B7B000D00000202DE9FE43FE480078FE490978BC
:10B7C000884205D1FD480078FD490978884203D0B8
:10B7D0000020FC49087010E0FA48007850B9FA4897
:10B7E000007818B90120F749087006E00020F549F3
:10B7F000087002E00020F3490870F148007813282F
:10B800007ED2DFE800F07D0A0B0C0D5994959697D7
:10B81000EE98999A9BEDECEBEA0000BF00BF00BFE9
:10B820000520FFF7B3FAE748007840B9E7490D78FB
:10B8300005EBD5714810E6A20621FFF71FFC202476
:10B84000012023465F22214600900020FFF738FBAD
:10B85000641C012023465F22214600900020FFF750
:10B860002FFB641C0120FFF791FAD8480078FBF702
:10B87000DDFC07460022D84BFBF766FC0546FBF7CC
:10B88000E2FC00F0FF09D5A228214846FFF7F6FBAD
:10B89000CE480078FBF7CAFC07460022D34BFBF7E3
:10B8A00053FC0546FBF7CFFC00F0FF09D0A2322184
:10B8B0004846FFF7E3FB52E20520FFF767FAC3496A
:10B8C0000D7805EBD5714810C1A20621FFF7D6FB14
:10B8D0002024012023465F22214600900020FFF70C
:10B8E000EFFA641C012023465F22214600900020CD
:10B8F000FFF7E6FA641C0220FFF748FABF4800E0B1
:10B900002CE2007848B9B1490D7805EBD5714810A3
:10B91000BBA22821FFF7B2FB08E0AC490D7805EB8C
:10B92000D5714810B9A22821FFF7A8FB17E200BF84
:10B9300000BF00BF00BF00BF00BF00BF0520FFF772
:10B9400025FAB5A206210020FFF798FB9D48007854
:10B9500000284CD1B1488278B1A1B248FDF7B8FABD
:10B96000B04A06212320FFF789FB95480078062876
:10B970000FD09348007807280BD09148007808280A
:10B9800007D08F4800780B2803D08D4800780C280A
:10B990002DD18B480078062807D0894800780728E1
:10B9A00003D087480078082805D19F4A06215020F7
:10B9B000FFF788FB1BE09D4800889D490988884265
:10B9C00015D0964880789949098888420ADB994AB7
:10B9D00006214E20FFF776FB09E0B2E19FE09BE0F5
:10B9E00043E041E0944A06214E20FFF76BFB012023
:10B9F000FFF7CCF991A20D214420FFF73FFB9048BF
:10BA0000C07B012801D18FA000E08FA002468FA14A
:10BA10008448FDF75DFA834A12214820FFF72EFB88
:10BA20000520FFF7B3F92024012023465F22214699
:10BA300000900020FFF744FA641C012023465F2297
:10BA4000214600900020FFF73BFA641C0120FFF71D
:10BA50009DF97FA228210020FFF710FB81A232214F
:10BA60000020FFF70BFB7AE100BF0520FFF78EF9FE
:10BA70006A48827880A16B48FDF72AFA53490D780D
:10BA800005EBD5714810674A0621FFF7F7FA012048
:10BA9000FFF77CF969A20F215520FFF7EFFA6848FC
:10BAA000C07B012801D167A000E067A0024667A122
:10BAB0005C48FDF70DFA5B4A14215920FFF7DEFAC6
:10BAC0000220FFF763F94D48007848B93F490D78E7
:10BAD00005EBD57148104AA22821FFF7CFFA08E0FC
:10BAE0003A490D7805EBD571481048A22821FFF797
:10BAF000C5FA2024012023465F2221460090002021
:10BB0000FFF7DEF9641C012023465F2221460090E6
:10BB10000020FFF7D5F922E100F06CF91FE10120C8
:10BB2000FFF734F9042429490D7805EBD571481045
:10BB300053A22146FFF7A2FA554800782044C4B228
:10BB40000520FFF723F93E48807CFF2805D151A24C
:10BB50003EA102A8FDF7BCF905E03948827C30A17E
:10BB600002A8FDF7B5F93648C07CFF2805D149A2E7
:10BB700036A101A8FDF7ACF905E03148C27C28A147
:10BB800001A8FDF7A5F901AB02AA43A12548FDF7DD
:10BB90009FF9A01CC4B20D490D7805EBD571481072
:10BBA000204A2146FFF76AFA0120FFF7EFF8E01D6F
:10BBB000C1B275E0D0000020CF000020D4000020EA
:10BBC00047000020D2000020A3000020E800002051
:10BBD000204F4646200000000000F83F53656E7479
:10BBE000204F464620636F6465000000000004405B
:10BBF00066726F6D2052656D6F746500580000208D
:10BC000020204C6561726E65642020002020204554
:10BC100072726F72202020004F4E0000220200201E
:10BC200025326400F020002026EF00086400002088
:10BC30006600002086EF000856EF00082E00000086
:10BC4000320C002046000000430000002573000075
:10BC500041646A75737420536574706F696E743BC8
:10BC60000000000053656E642052656D6F7465209E
:10BC7000636F6465000000004F4E2F2532640000A2
:10BC80002053657474696E672052616E6765200089
:10BC9000E90000202D2D000025737E257300000093
:10BCA000AFF268025420FFF7E9F93048C07B012861
:10BCB00002D1AFF2700001E0AFF274000246AFF2C1
:10BCC00074012B48FDF704F904F10C00C1B2284AB5
:10BCD0005820FFF7D3F90520FFF758F825480078DA
:10BCE0002044C4B2012023465F2221460090002058
:10BCF000FFF7E6F8601CC4B2012023465F2221460C
:10BD000000900020FFF7DCF8601CC4B20120FFF7B0
:10BD10003DF8A01CC4B218A221461B480078FFF7CA
:10BD2000ADF9144800782044C4B2A01CC4B216492E
:10BD30000D7805EBD571481014A22146FFF79EF946
:10BD40000DE00520FFF722F80F490D7805EBD571BE
:10BD5000481012A21421FFF791F900BF00BF00BFE5
:10BD60001048007810490870BDE8FE83320C0020AE
:10BD7000F0200020E900002020205072657373201D
:10BD8000456E746572202000E800002020202020ED
:10BD9000546F205361766520202020005361766522
:10BDA0006400000047000020D400002010B50220ED
:10BDB000FEF7ECFF07A20C210020FFF75FF909490D
:10BDC0000C7804EBD471481007A22421FFF756F930
:10BDD00010BD000020202044657669636520202086
:10BDE00000000000E800002020206F66666C696E8D
:10BDF000652020002DE9F0410220FEF7C7FF17491A
:10BE0000097801EB4101C8B215A20421FFF736F908
:10BE100012480078FBF70AFA05460022124BFBF79E
:10BE200093F90746FBF70FFAC4B210A21821204677
:10BE3000FFF724F909480078FBF7F8F905460022D6
:10BE40000D4BFBF781F90746FBF7FDF9C4B20BA2D6
:10BE50002C212046FFF712F9BDE8F081E800002010
:10BE60004D415820323400000000F83F5365747093
:10BE70006F696E74730000000000044052656163D6
:10BE8000686564002DE9F0474FF000090220FEF7D5
:10BE90007DFF10480078FBF7C9F9074600220E4BDA
:10BEA000FBF752F90546FBF7CEF9C4B20BA21221FB
:10BEB0002046FFF7E3F80220FEF768FF05490978FE
:10BEC00001EB4101C8B207A22621FFF7D7F8BDE870
:10BED000F0870000E800002000000C404152532D84
:10BEE0003100000056455220312E362E3900000018
:10BEF0002DE9FE43D448007803287DD1D248C07B89
:10BF0000D149097D884278D104240120FEF73EFF03
:10BF1000CE490D7805EBD5714810CDA22146FFF72B
:10BF2000ADF8CF4800782044C4B20520FEF72EFFBC
:10BF3000C548807CFF2805D1CAA2CBA102A8FCF786
:10BF4000C7FF05E0C048827CC8A102A8FCF7C0FF7B
:10BF5000BD48C07CFF2805D1C2A2C3A101A8FCF73F
:10BF6000B7FF05E0B848C27CC0A101A8FCF7B0FF4C
:10BF700001AB02AABEA1C048FCF7AAFFA01CC4B234
:10BF8000B2490D7805EBD5714810BB4A2146FFF741
:10BF900075F80120FEF7FAFEE01DC1B2B7A25420E9
:10BFA000FFF76CF8A848C07B012801D1B4A000E0DD
:10BFB000B4A00246ACA1B048FCF78AFF04F10C0023
:10BFC000C1B2AD4A5820FFF759F80520FEF7DEFE52
:10BFD000A34800782044C4B2A01EC4B20120234666
:10BFE0005F22214600900020FEF76AFF601CC4B269
:10BFF000012023465F2201E0EBE00FE021460090A4
:10C000000020FEF75DFF601CC4B2012023465F22C2
:10C01000214600900020FEF753FFABE08A48407CA9
:10C02000012870D10424FEF7B1FE88490D7805EB94
:10C03000D571481086A22146FFF720F8884800787D
:10C040002044C4B20520FEF7A1FE86A286A102A864
:10C05000FCF73EFF83A284A101A8FCF739FF01ABE6
:10C0600002AA83A18448FCF733FFA01CC4B277491D
:10C070000D7805EBD57148107F4A2146FEF7FEFF8B
:10C080000120FEF783FEE01DC1B27CA25420FEF722
:10C09000F5FF6D48C07B012801D179A000E079A0AF
:10C0A000024671A17448FCF713FF04F10C00C1B201
:10C0B000714A5820FEF7E2FF0520FEF767FE684848
:10C0C00000782044C4B2A01EC4B2012023465F22DF
:10C0D000214600900020FEF7F3FE601CC4B2012050
:10C0E00023465F22214600900020FEF7E9FE601CF7
:10C0F000C4B2012023465F22214600900020FEF7B3
:10C10000DFFE37E0FFE702240220FEF73FFE4F4943
:10C110000D7805EBD57148105BA22146FEF7AEFF06
:10C120004F4800782044C4B2A01CC4B247490D78DF
:10C1300005EBD571481057A22146FEF79FFF242436
:10C14000012023465F22214600900020FEF7B8FE22
:10C15000641C012023465F22214600900020FEF748
:10C16000AFFE641C012023465F2221460090002080
:10C17000FEF7A6FE0120FEF709FE2A24E41C48A2D1
:10C1800021460020FEF77AFF621ED1B22F4A1278B4
:10C1900002EB42025200121FD0B2464AFEF771FD76
:10C1A0002F4800780444E01CC4B228480078FBF70C
:10C1B0003DF807460022404BFAF7C6FF0546FBF75D
:10C1C00042F800F0FF093DA221464846FEF756FF1F
:10C1D00037E01D480078022822D10424FEF7D6FD5E
:10C1E00039A221460020FEF749FF1D48007820446F
:10C1F000C4B2E01CC4B238A221460020FEF73EFFC4
:10C20000174800782044C4B2E01CC4B20F490D782E
:10C2100005EBD571481034A22146FEF72FFF10E040
:10C220000220FEF7B3FD33A20C210020FEF726FF0B
:10C2300006490D7805EBD571481032A22421FEF78E
:10C240001DFFBDE8FE830000320C0020E800002046
:10C250002053657474696E672052616E67652000B3
:10C26000E90000202D2D0000257300002532640018
:10C2700025737E2573000000F02000202E000000B2
:10C28000460000004300000054656D7020466F7248
:10C290006D6174002020204572726F722020200092
:10C2A0005072657373202020746F204C6561726E2C
:10C2B00000000000B6EF00080000044052656D6FFA
:10C2C000746520436F646500506C65617365207010
:10C2D00072657373000000002041646472657373BB
:10C2E000696E672000000000202020206B65792007
:10C2F00020202000202020446576696365202020CE
:10C300000000000020206F66666C696E65202000CA
:10C3100010B533480078FF281FD13248407CA8B9B7
:10C320003048007D2F49C97B884207D100202E4923
:10C33000087000212D48FFF727FA0EE001202A4956
:10C34000087000212A48FFF71FFA06E0012026495D
:10C35000087000212648FFF717FA2348007820B11B
:10C3600001282FD0022837D131E01E480078032859
:10C3700020D11C48407CA8B91A48007D1949C97BC6
:10C38000884207D100201849087000211748FFF79C
:10C39000FBF916E001201449087000211448FFF74A
:10C3A000F3F90EE001201049087000211048FFF752
:10C3B000EBF906E000200C49087000210B48FFF75C
:10C3C000E3F90AE000210A48FFF7DEF905E0002161
:10C3D0000848FFF7D9F900E000BF00BF10BD00001A
:10C3E000D1000020320C0020CF00002089B30008CB
:10C3F000F1BE0008B5B7000800B5FF201C49087061
:10C400001C49087000201C4908701C4908704870BD
:10C41000A1F84E05A1F86E0AC8850120087440F203
:10C420007E2200211648FEF7A3FF40F27E22002163
:10C430001448FEF79DFF40F27E2200210F48323063
:10C44000FEF796FF07201049087000200F4908707A
:10C4500004200F4908700F49087000200E49087029
:10C460000E48007840F020000C49087000BD000024
:10C47000D10000201A00002062000020320C0020B1
:10C4800084110020A4160020480000204400002051
:10C4900060000020610000206A0000205900002098
:10C4A0002DE9F05F82460E464FF0000BD846012E74
:10C4B00007D10AEB8A004FF4A06101EB002085B29E
:10C4C00000E000250027D5E04FF0000BD846594684
:10C4D0000BF1010B05EB811188B240226849FDF791
:10C4E000C3FC67488078674981F806056448C078CE
:10C4F0008870634840796249097940EA01206149BE
:10C5000008805F48C0795E49897940EA01205D4929
:10C51000A1F804055A4840785949097840EA0120B1
:10C5200045F2AA51884208D1564890F806050128DC
:10C530000CD0544890F8060540B13220FDF712FCAB
:10C54000FDF71CFE3220FDF70DFC91E04D48008800
:10C55000082805DB4B48008840F27E21884208DB32
:10C560003220FDF7FFFBFDF709FE3220FDF7FAFB55
:10C570007EE0012E26D1434890F80605012810D10F
:10C5800040488078322803DB3E488078632819DDF4
:10C590003220FDF7E7FBFDF7F1FD3220FDF7E2FB6E
:10C5A00066E0384880780A2803DB364880783228ED
:10C5B00008DD3220FDF7D6FBFDF7E0FD3220FDF768
:10C5C000D1FB55E008240FE02D49601C085C095D93
:10C5D00040EA01224046411C1FFA81F82949091D01
:10C5E00021F81020A01CC4B2402CEDDB00BF59463E
:10C5F0004A1C02F0FF0B05EB811188B24022204952
:10C60000FDF732FC002414E01D49601C085C095D44
:10C6100040EA01224146481C1FFA80F81948001DD3
:10C6200020F81120A01CC4B240F27E20804500DB1F
:10C6300002E0402CE8DBDAE7124800884FF6FF7290
:10C6400002EA40010F48001DFDF738FB81460D4806
:10C65000B0F80415494502D10020BDE8F09F322012
:10C66000FDF780FBFDF78AFD3220FDF77BFB00BF65
:10C67000781CC7B2052F7FF727AF0120EDE7000038
:10C680000E2100202A07002010B500210846FFF7E0
:10C6900007FF78B9254800882549A1F84E052348A9
:10C6A0000288011D234800F06FF9204890F8060524
:10C6B0001F490875002427E001212046FFF7F0FEFE
:10C6C000F8B91B48007D194991F80615884219D11F
:10C6D000164881781648163001556CB91348807891
:10C6E0001349887411480088A1F86E0A0F4802881F
:10C6F000011D114800F048F90C4880780C49C874B5
:10C7000000E003E0601CC4B2182CD5DB00BF084871
:10C71000447534B9FF2006498874C87401204874F0
:10C7200010BD00200249487400BFF9E72A07002025
:10C73000320C002084110020A416002010B5002423
:10C740000120224908702248006820F47020204906
:10C7500008600846006840F40020086000BF4FF4FD
:10C7600000601B4910310860FDF756FC6006040E9E
:10C770004FF4006016490C310860FDF74DFC144879
:10C78000001D006800F4805008B144F001040F4817
:10C7900000784006000E0D49087008460078002811
:10C7A000DDD14FF400600A4910310860FDF734FC18
:10C7B0000748006820F470200549086008460068B2
:10C7C00040F440300860204610BD000042000020C8
:10C7D0000408014010B51748006820F4702015497E
:10C7E00008600846006840F440300860C8141149E9
:10C7F000103108604000091F0860FDF70DFC4FF480
:10C8000000600C490C310860FDF706FC4FF4006035
:10C81000084910310860FDF7FFFB0648006820F466
:10C820007020044908600846006840F40020086051
:10C8300010BD00000408014010B51948006820F43C
:10C840007020174908600846006840F440300860CE
:10C85000C814134910310860FDF7DEFB4FF4805017
:10C860000F4910310860FDF7D7FB4FF400600C4909
:10C870000C310860FDF7D0FB4FF40060084910311F
:10C880000860FDF7C9FB0648006820F470200449E1
:10C8900008600846006840F40020086010BD0000F1
:10C8A000040801402DE9F04107468024354800681E
:10C8B00020F47020334908600846006840F4403096
:10C8C000086000BF4FF400602E4910310860FDF78A
:10C8D000A3FB07EA040028B14FF4805029490C312A
:10C8E000086004E04FF48050264910310860FDF7DD
:10C8F00093FB4FF4006023490C3108606410FDF78E
:10C900008BFB002CDED14FF400601E491031086013
:10C910001C48006820F470201A4908600846006826
:10C9200040F400200860FDF777FB4FF400601549E4
:10C930000C310860642600BFFDF76EFB701EC0B2AC
:10C94000060006D00F48001D0068C0F30030002824
:10C95000F2D10C48001D0068C0F300354FF40060B0
:10C960000849103108600748006820F47020054924
:10C9700008600846006840F4403008602846BDE87A
:10C98000F08100000408014070B503460C4603E046
:10C9900034F8025B23F8025B1500A2F10106B2B283
:10C9A000F6D170BD10B504464048007802287CD10D
:10C9B0003F480078062803D03D4800780B2874D102
:10C9C0003B48007806280DD13A48007830B90A2053
:10C9D0003949087001203749087009E005203649B7
:10C9E000087005E0002033490870FF2032490870C4
:10C9F0002F48007806282DD1012C15D12F4880789A
:10CA0000401C2E498870084680782D490988884244
:10CA100005DC2A4880782B49098888423BDA294876
:10CA200000782649887036E024488078401E2349E3
:10CA300088700846807822490988884205DC1F48AA
:10CA4000807820490988884225DA1D4800781B49EA
:10CA5000887020E0012C0FD118488078401C1749BD
:10CA600088700846807816490988884213DB144884
:10CA70000078124988700EE010488078401E0F49F7
:10CA80008870084680780F490988884203DC0D4881
:10CA900000780A49887000200B49087000210B4873
:10CAA000FEF772FE1E20FDF725F910BDCF00002015
:10CAB00047000020A3000020CD000020220200201B
:10CAC0006400002066000020D2000020B5B70008F6
:10CAD00010B586B0044601940020ADF80800ADF80A
:10CAE0000A00ADF80C00ADF810000C20ADF80E00F7
:10CAF00001210420FBF70EF900214FF48040FBF7E1
:10CB000019F901218803FBF705F94FF40070ADF81E
:10CB1000140018208DF8170003208DF8160005A9C1
:10CB20001548FAF7F5FE4FF48060ADF814000420C4
:10CB30008DF8170005A91048FAF7EAFE01A90F4879
:10CB4000FCF754F925208DF8000003208DF8010032
:10CB50008DF8020001208DF803006846FBF766F8A7
:10CB6000012240F225510548FCF71BF90121034839
:10CB7000FCF7FEF806B010BD000801400038014087
:10CB800070B505460E4680211148FAF7A4FF00242F
:10CB90000CE000BF40210F48FCF7F6F80028F9D060
:10CBA000295D0C48FCF78EF9601CC4B2B442F0DB7E
:10CBB00000BF40210748FCF7E7F80028F9D08021A2
:10CBC0000348FAF786FF00200349086070BD0000A3
:10CBD00000080140003801401C00002070B500250D
:10CBE00000240F4E00BF17E0B02141EAE400FAF73D
:10CBF000B7FF1120FAF7B4FF0220FAF7B1FF0025C2
:10CC000005E016F8010BFAF7D9FF681CC5B25F2DD5
:10CC1000F7DD04F10800C4B2402CE5DD70BD000072
:10CC20005C2100202DE9F047804689460024A24679
:10CC3000B9F1010F07D108EB88004FF4A06101EBB7
:10CC4000002086B200E000265F4800884FF6FF72A1
:10CC500002EA40015C48001DFDF730F85A49A1F88E
:10CC600004050027AAE04FF0000A00245520574988
:10CC70000870AA204870544890F8060588705248F9
:10CC80008078C87050480088001208714E480078BB
:10CC900048714D48B0F80405001288714A4890F870
:10CCA0000405C871082515E04748001D30F8140038
:10CCB00002122846691CCDB244490A542046611C20
:10CCC0008CB24149091D11F810202846691CCDB2CB
:10CCD0003E490A54402DE7DB51464A1C02F0FF0A48
:10CCE00006EB811188B240223849FDF7E5F80025AE
:10CCF00022E03548001D30F8140002122846691C55
:10CD0000CDB232490A543048001D10F8142028468C
:10CD1000691CCDB22D490A54402D0BDB51464A1CEB
:10CD200002F0FF0A06EB811188B240222749FDF785
:10CD3000C3F80025601C84B240F27E208442D8DB18
:10CD400049464046FFF7ACFBE0B91F480088204940
:10CD5000098888420DD11C4880781D49897888420D
:10CD600007D1194890F80605194991F80615884227
:10CD700011D00A20FCF7F6FFFDF700FA3220FCF78D
:10CD8000F1FF19E00A20FCF7EDFFFDF7F7F932207B
:10CD9000FCF7E8FF10E00C48B0F804050C49B1F8C6
:10CDA0000415884207D1084890F806050949087516
:10CDB0000020BDE8F08700BF781CC7B2052F7FF7C1
:10CDC00052AF0120F5E70000220200200E210020D2
:10CDD0002A070020320C002070B5034601F0070638
:10CDE0000125B540ECB2CD1005EB45050A4E06EB2A
:10CDF0004515E85C012A01D1204305E00AB9A043AA
:10CE000002E0022A00D16040CD1005EB4505024E3C
:10CE100006EB4515E85470BD5C2100203C0F480D21
:10CE20008C0A6C075E01000000010203040500C1CA
:10CE3000814001C0804101C0804100C1814001C0EA
:10CE4000804100C1814000C1814001C0804101C0DA
:10CE5000804100C1814000C1814001C0804100C1CA
:10CE6000814001C0804101C0804100C1814001C0BA
:10CE7000804100C1814000C1814001C0804100C1AA
:10CE8000814001C0804101C0804100C1814000C19A
:10CE9000814001C0804101C0804100C1814001C08A
:10CEA000804100C1814000C1814001C0804101C07A
:10CEB000804100C1814000C1814001C0804100C16A
:10CEC000814001C0804101C0804100C1814000C15A
:10CED000814001C0804101C0804100C1814001C04A
:10CEE000804100C1814000C1814001C0804100C13A
:10CEF000814001C0804101C0804100C1814001C02A
:10CF0000804100C1814000C1814001C0804101C019
:10CF1000804100C1814000C1814001C0804100C109
:10CF2000814001C0804101C0804100C1814000C0FA
:10CF3000C101C30302C2C60607C705C5C404CC0CA1
:10CF40000DCD0FCFCE0E0ACACB0BC90908C8D81811
:10CF500019D91BDBDA1A1EDEDF1FDD1D1CDC14D421
:10CF6000D515D71716D6D21213D311D1D010F03051
:10CF700031F133F3F23236F6F737F53534F43CFC61
:10CF8000FD3DFF3F3EFEFA3A3BFB39F9F83828E811
:10CF9000E929EB2B2AEAEE2E2FEF2DEDEC2CE424E1
:10CFA00025E527E7E62622E2E323E12120E0A06051
:10CFB00061A163A3A26266A6A767A56564A46CAC21
:10CFC000AD6DAF6F6EAEAA6A6BAB69A9A86878B891
:10CFD000B979BB7B7ABABE7E7FBF7DBDBC7CB474A1
:10CFE00075B577B7B67672B2B373B17170B0509051
:10CFF00091519353529296565797559594549C5CE1
:10D000005D9D5F9F9E5E5A9A9B5B99595898884890
:10D0100049894B8B8A4A4E8E8F4F8D4D4C8C448460
:10D020008545874746868242438341818040000090
:10D0300000000000000000000000000000000000F0
:10D04000183C3C3C18181800181800000000006636
:10D0500066662400000000000000000000000000E0
:10D06000006C6CFE6C6C6CFE6C6C000000001818A0
:10D070007CC6C2C07C060686C67C1818000000006C
:10D080000000C2C60C183060C68600000000000018
:10D09000386C6C3876DCCCCCCC76000000000030EC
:10D0A00030306000000000000000000000000000C0
:10D0B0000C18303030303030180C00000000000008
:10D0C00030180C0C0C0C0C0C183000000000000088
:10D0D000000000663CFF3C6600000000000000000D
:10D0E00000000018187E1818000000000000000062
:10D0F00000000000000000181818300000000000B8
:10D100000000000000FE0000000000000000000021
:10D1100000000000000000001818000000000000DF
:10D12000000002060C183060C08000000000000003
:10D13000386CC6C6C6C6C6C66C3800000000000003
:10D140001838781818181818187E00000000000009
:10D150007CC6060C183060C0C6FE0000000000004F
:10D160007CC606063C060606C67C000000000000E1
:10D170000C1C3C6CCCFE0C0C0C1E000000000000D3
:10D18000FEC0C0C0FC060606C67C00000000000011
:10D190003860C0C0FCC6C6C6C67C000000000000E7
:10D1A000FEC606060C1830303030000000000000CB
:10D1B0007CC6C6C67CC6C6C6C67C00000000000091
:10D1C0007CC6C6C67E0606060C780000000000007D
:10D1D00000001818000000181800000000000000EF
:10D1E00000001818000000181830000000000000AF
:10D1F00000060C18306030180C060000000000001B
:10D200000000007E00007E00000000000000000022
:10D21000006030180C060C183060000000000000A0
:10D220007CC6C60C18181800181800000000000072
:10D23000007CC6C6DEDEDEDCC07C00000000000034
:10D2400010386CC6C6FEC6C6C6C600000000000088
:10D25000FC6666667C66666666FC00000000000090
:10D260003C66C2C0C0C0C0C2663C000000000000F6
:10D27000F86C6666666666666CF800000000000082
:10D28000FE6662687868606266FE0000000000006A
:10D29000FE6662687868606060F000000000000070
:10D2A0003C66C2C0C0DEC6C6663A00000000000090
:10D2B000C6C6C6C6FEC6C6C6C6C60000000000007A
:10D2C0003C18181818181818183C00000000000026
:10D2D0001E0C0C0C0C0CCCCCCC7800000000000018
:10D2E000E666666C78786C6666E600000000000012
:10D2F000F06060606060606266FE00000000000038
:10D30000C6EEFEFED6C6C6C6C6C6000000000000B9
:10D31000C6E6F6FEDECEC6C6C6C6000000000000A9
:10D320007CC6C6C6C6C6C6C6C67C000000000000D5
:10D33000FC6666667C60606060F0000000000000D3
:10D340007CC6C6C6C6C6C6D6DE7C0C0E0000000073
:10D35000FC6666667C6C666666E60000000000009F
:10D360007CC6C660380C06C6C67C00000000000003
:10D370007E7E5A1818181818183C0000000000008B
:10D38000C6C6C6C6C6C6C6C6C67C0000000000002B
:10D39000C6C6C6C6C6C6C66C38100000000000006F
:10D3A000C6C6C6C6D6D6D6FEEE6C0000000000008B
:10D3B000C6C66C7C38387C6CC6C600000000000015
:10D3C000666666663C181818183C000000000000ED
:10D3D000FEC6860C183060C2C6FE000000000000C9
:10D3E0003C30303030303030303C00000000000045
:10D3F0000080C0E070381C0E060200000000000033
:10D400003C0C0C0C0C0C0C0C0C3C000000001038FC
:10D410006CC60000000000000000000000000000DA
:10D420000000000000000000000000FF00000030CD
:10D43000180C0000000000000000000000000000C8
:10D44000000000780C7CCCCCCC7600000000000002
:10D45000E06060786C666666667C00000000000034
:10D460000000007CC6C0C0C0C67C000000000000F8
:10D470001C0C0C3C6CCCCCCCCC760000000000002A
:10D480000000007CC6FEC0C0C67C0000000000009A
:10D490001C36323078303030307800000000000028
:10D4A00000000076CCCCCCCCCC7C0CCC780000003E
:10D4B000E060606C7666666666E60000000000006C
:10D4C0001818003818181818183C00000000000040
:10D4D0000606000E06060606060666663C00000006
:10D4E000E06060666C78786C66E600000000000022
:10D4F0003818181818181818183C000000000000F8
:10D50000000000ECFED6D6D6D6C600000000000013
:10D51000000000DC666666666666000000000000CB
:10D520000000007CC6C6C6C6C67C00000000000025
:10D53000000000DC66666666667C6060F0000000E5
:10D5400000000076CCCCCCCCCC7C0C0C1E000000B7
:10D55000000000DC7666606060F000000000000003
:10D560000000007CC660380CC67C00000000000093
:10D57000103030FC30303030361C0000000000002D
:10D58000000000CCCCCCCCCCCC760000000000005D
:10D59000000000C6C6C6C6C66C3800000000000009
:10D5A000000000C6C6D6D6D6FE6C00000000000003
:10D5B000000000C66C3838386CC60000000000005F
:10D5C000000000C6C6C6C6C6C67E060CF80000002F
:10D5D000000000FECC183060C6FE00000000000015
:10D5E0000E18181870181818180E00000000000007
:10D5F000181818181818181818180000000000003B
:10D60000701818180E18181818700000000000760E
:10D61000DC0000000000000000000000000000002E
:10D620001C300000000000000000000000000000AE
:10D630007018000000000000000000000000001052
:10D64000386C00000000000000000000000000C670
:10D65000C60000000000000000000000000000768E
:10D66000DC000000000000000000000000000000DE
:10D670000000003818181818183C000000000000BE
:10D68000386C6C6C786C6666666C60C00000102844
:10D6900010007CC6C6FEC6C6C6C60000000000302C
:10D6A000483000780C7CCCCCCC7600000000000028
:10D6B0001E7AD8D8D8FED8D8DADE000000000000E4
:10D6C000FC666666F6F6666666FC00000000000012
:10D6D000F0607C666666667C60F00000000000001A
:10D6E000000000CC323E70B0B26C000000000000C0
:10D6F000D060B0187CC6C6C6C67C00000000000022
:10D70000E06060786C6C786060F000000000000001
:10D710007CC6CECED6D6E6E6C67C00000000000071
:10D720000000003A44CED6E644B8000000000000F5
:10D7300000386CC6C6FEC6C6C6C6000000000000A3
:10D7400000FE66626878686266FE00000000000005
:10D75000003C181818181818183C000000000000A9
:10D76000007CC6C6C6C6C6C6C67C00000000000057
:10D7700000C6C6C6C6C6C6C6C67C000000000000FD
:10D7800000C6E6F6FEDECEC6C6C6000000000000FB
:10D790001818001818183C3C3C1800000000000045
:10D7A00030300030303060C6C67C000000001C30D5
:10D7B00000000000000000000000000000007018E1
:10D7C0000000000000000000000000000000386CB5
:10D7D0000000000000000000000000000000C6C6BD
:10D7E000000000000000000000000000000076DCE7
:10D7F0000000000000000000000000000000000029
:10D8000000000000000000000000183000000000D0
:10D810000000000000000000000000000000000008
:10D820000010107CD0D0D0D0D67C101000000000AA
:10D830001C30303078303030325C000000000000A6
:10D840000000423C24243C42000000000000000094
:10D85000663C187E18187E1818180000000000009A
:10D8600018181818000018181818000000000000F8
:10D870003C6460384444380C4C780000000000C61A
:10D88000C6000000000000000000000000000000D2
:10D8900000007E425A5E5A427E00000000000000F6
:10D8A0007008788888740000000000000000000004
:10D8B000000000366CD86C3600000000000000004C
:10D8C0000000000000FC0404000000000000000054
:10D8D00000000000007C00000000000000000000CC
:10D8E00000007C4454444C547C0000000000FE00C6
:10D8F00000000000000000000000000000000070B8
:10D90000D888D8700000000000000000000000006F
:10D91000000010107C1010007C0000000000788CCB
:10D920000C183060FC000000000000000000788C43
:10D930000C780C8C78000000000000000000000E45
:10D94000182000000000000000000000000000009F
:10D950000000006666666666667C6060C000000067
:10D960007ED4D4D474141414143E000000000000BB
:10D97000000000003838380000000000000060E0BF
:10D9800060606060F0000000000000000000000027
:10D990003C6666663C0000000000000000000000DD
:10D9A000000000D86C366CD80000000000000000B9
:10D9B00040C0444810244C941E04000000000000A5
:10D9C00040C04448102C5284081E00000000000093
:10D9D000C0204428D0244C941E0400000000000005
:10D9E000000000663C183C660000000000000000DB
:10D9F00000001818007E0018180000000000000049
:10DA00000000000818387FFF7F3818080000000069
:10DA100000000010181CFEFFFE1C18100000000083
:10DA20000000000010387CFE383838380000000054
:10DA30000000000038383838FE7C38100000000044
:10DA4000000606060616367EFE7C3010000000003A
:10DA500000000000030306060CCC7838000000002C
:10DA60000000000000002020202020002000484866
:10DA70004800000000005050F850F8505000207846
:10DA8000A07028F02000C0C81020409818006090B6
:10DA9000A040A89068006020400000000000102016
:10DAA0004040402010004020101010204000005046
:10DAB00020F820500000002020F820200000000066
:10DAC000000000602040000000F80000000000009E
:10DAD0000000006060000008102040800000708896
:10DAE00098A8C888700020602020202070007088CE
:10DAF00008304080F80070880830088870001030C6
:10DB00005090F8101000F880F0080888700030403D
:10DB100080F088887000F80810204040400070882D
:10DB200088708888700070888878081060000060AD
:10DB30006000606000000000606000602040102015
:10DB40004080402010000000F800F80000008040F5
:10DB5000201020408000708808102000200070886D
:10DB60000868A8A87000708888F888888800F088FD
:10DB700088F08888F0007088808080887000E0904D
:10DB800088888890E000F88080F08080F800F88035
:10DB900080F08080800070888080988878008888F5
:10DBA00088F8888888007020202020207000381095
:10DBB0001010109060008890A0C0A0908800808015
:10DBC00080808080F80088D8A8A888888800888805
:10DBD000C8A8988888007088888888887000F0882D
:10DBE00088F08080800070888888A8906800F0881D
:10DBF00088F0A09088007088807008887000F820F5
:10DC000020202020200088888888888870008888C4
:10DC1000888888502000888888A8A8A8500088880C
:10DC20005020508888008888885020202000F808DC
:10DC300010204080F800704040404040700000805C
:10DC400040201008000070101010101070002050BC
:10DC500088000000000000000000000000F84020E4
:10DC600010000000000000007008788878008080B4
:10DC7000B0C88888F00000007080808870000808B4
:10DC800068988888780000007088F88070003048B4
:10DC900040E040404000000078888878087080802C
:10DCA000B0C8888888002000602020207000100004
:10DCB000301010109060808090A0C0A09000602074
:10DCC0002020202070000000D0A888888800000054
:10DCD000B0C88888880000007088888870000000BC
:10DCE000F08888F080800000788888780808000034
:10DCF000B0C880808000000078807008F00040404C
:10DD0000E0404048300000008888889868000000A3
:10DD100088888850200000008888A8A8500000004B
:10DD2000885020508800000088888878087000009B
:10DD3000F8102040F8001020204020201000202063
:10DD4000202020202000402020102020400068902B
:10DD500000000000000000000000000000000000C3
:10DD600000000000000000000000000000000000B3
:10DD700000000000000000000000000000000000A3
:10DD8000000000000000000000000000000038005B
:10DD900038003800380038003800380038003800C3
:10DDA00010001000000038003800380000000000AB
:10DDB0000000000000000000000000000000738070
:10DDC0007380738073807380000000000000000087
:10DDD0000000000000000000000000000000000043
:10DDE00000000000000000000000000000000C60C7
:10DDF0000C600C6018C0FFF0FFF018C039C0318013
:10DE0000FFF0FFF0318073806300630000000000CA
:10DE100000000000000000000000000006001F805D
:10DE20003FC076E076E076007E003F001FC007E04E
:10DE300006E006E076E076E03FC01F8006000600C0
:10DE400000000000000000000000000000003C187E
:10DE50007E3866306630666066607EC03CC0019E7B
:10DE600001BF03B3033303330633063F0C1E000028
:10DE7000000000000000000000000000000007801B
:10DE80000FC01CE01CE01EE00FC00F801F803F9CF5
:10DE900071FC71F870F079FC3FFE1F8C00000000EF
:10DEA0000000000000000000000000000000700002
:10DEB00070007000700070000000000000000000A2
:10DEC0000000000000000000000000000000000052
:10DED00000000000000000000000000000000C0036
:10DEE00018001800380038007000700070007000D2
:10DEF00070007000700070003000380038001800AA
:10DF000018000C000000000000000000000060008D
:10DF100030003000380038001C001C001C001C00C1
:10DF20001C001C001C001C001800380038003000C9
:10DF30003000600000000000000000000000180039
:10DF40001800DB00FF001C003C00660024000000FD
:10DF500000000000000000000000000000000000C1
:10DF600000000000000000000000000000000000B1
:10DF7000000007000700070007007FF07FF07FF038
:10DF80000700070007000700000000000000000075
:10DF90000000000000000000000000000000000081
:10DFA0000000000000000000000000000000000071
:10DFB00000000000000070007000700010003000D1
:10DFC00060000000000000000000000000000000F1
:10DFD00000000000000000000000000000007E00C3
:10DFE0007E007E0000000000000000000000000035
:10DFF0000000000000000000000000000000000021
:10E000000000000000000000000000000000000010
:10E0100000000000000070007000700000000000B0
:10E0200000000000000000000000000000000C00E4
:10E030000C001800180018003800300030003000C4
:10E040006000600060006000C000C00000000000D0
:10E0500000000000000000000000000000000F00B1
:10E060003FC039C070E070E070E070E070E070E0D8
:10E0700070E070E070E039C03FC00F0000000000A9
:10E08000000000000000000000000000000003800D
:10E09000038007801F803F803B80238003800380B4
:10E0A000038003800380038003800380000000005E
:10E0B00000000000000000000000000000001F80C1
:10E0C0003FC079E070E000E000E001C003C00780DD
:10E0D0000F001E001C0038007FE07FE00000000001
:10E0E00000000000000000000000000000001F0011
:10E0F0003F8071C071C001C003C00F800F8001C09C
:10E1000000E000E070E079C03FC01F0000000000A8
:10E11000000000000000000000000000000003807C
:10E12000078007800F800F801B80338033806380DF
:10E13000C380FFE0FFE00380038003800000000055
:10E1400000000000000000000000000000001FC0F0
:10E150001FC03800380038003F807FC071E000E009
:10E1600000E000E070E079C03FC01F000000000048
:10E1700000000000000000000000000000000F8010
:10E180003FC039E07080700077807FC079C070E058
:10E1900070E070E070E039C03FC00F000000000088
:10E1A00000000000000000000000000000007FE010
:10E1B0007FE000E001C003800380070007000E003D
:10E1C0000E000E001C001C001C001C0000000000C3
:10E1D00000000000000000000000000000001F80A0
:10E1E0003FC079E070E070E039C01F801F8039C007
:10E1F00070E070E070E079E03FC01F800000000038
:10E2000000000000000000000000000000000F00FF
:10E210003FC039C070E070E070E070E039E03FE08E
:10E220001EE000E030E079C03FC01F0000000000A9
:10E2300000000000000000000000000000000000DE
:10E240000000000000003800380038000000000026
:10E250000000000000003800380038000000000016
:10E2600000000000000000000000000000000000AE
:10E2700000000000000038003800380000000000F6
:10E2800000000000000038003800380008001800C6
:10E29000300000000000000000000000000000004E
:10E2A0000000002000E007E01F807C0070007E007E
:10E2B0001FC007E000E00020000000000000000098
:10E2C000000000000000000000000000000000004E
:10E2D0000000000000007FE07FE07FE00000000021
:10E2E0007FE07FE07FE00000000000000000000011
:10E2F000000000000000000000000000000000001E
:10E300000000400070007E001F8003E000E007E096
:10E310003F807E0070004000000000000000000010
:10E3200000000000000000000000000000000F805E
:10E330003FE078F07070007000F001E003C00780EB
:10E3400007000700000007000700070000000000AA
:10E35000000000000000000000000000000003E0DA
:10E3600007F00F1C1C0E19CE33E63666666666662D
:10E37000666666666666666663FE31BE380E1C1C9F
:10E380000F3C07F003E0000000000000000007C0A1
:10E3900007C007C00EE00EE00EE01C701C7038389D
:10E3A0003FF83FF87FFC701C701CE00E000000007E
:10E3B00000000000000000000000000000003FE03E
:10E3C0003FF03FF83838383838383FF03FF03FF802
:10E3D000381C381C381C3FFC3FF83FF000000000A0
:10E3E000000000000000000000000000000007C066
:10E3F0001FF03FF83C3C781870007000700070000F
:10E40000700078183C3C3FF81FF007C00000000087
:10E4100000000000000000000000000000003FE0DD
:10E420003FF03FF83838383C381C381C381C381C52
:10E43000381C381C38383FF83FF03FC0000000005F
:10E4400000000000000000000000000000003FF895
:10E450003FF83FF83800380038003FF03FF03FF019
:10E460003800380038003FF83FF83FF8000000005F
:10E4700000000000000000000000000000003FF06D
:10E480003FF03FF03800380038003FE03FE03FE029
:10E49000380038003800380038003800000000002C
:10E4A000000000000000000000000000000003E089
:10E4B0000FF81FFC3C1E780C7000700070FE70FEA0
:10E4C00070FE380E3C1E1FFE0FFC03E00000000033
:10E4D0000000000000000000000000000000703894
:10E4E000703870387038703870387FF87FF87FF87F
:10E4F000703870387038703870387038000000002C
:10E500000000000000000000000000000000038088
:10E5100003800380038003800380038003800380E3
:10E5200003800380038003800380038000000000D9
:10E53000000000000000000000000000000001C01A
:10E5400001C001C001C001C001C001C001C001C0C3
:10E55000E1C0E1C0F1C07FC07F801E00000000006C
:10E560000000000000000000000000000000383C37
:10E57000387838F038E039C03B803FC03FC03EE0DB
:10E580003CE0387038383838381C381C000000003F
:10E590000000000000000000000000000000380043
:10E5A00038003800380038003800380038003800AB
:10E5B0003800380038003FF03FF03FF00000000026
:10E5C00000000000000000000000000000007C1FB0
:10E5D0007E3F7E3F76377637763777777777736704
:10E5E000736773E773E773E771C771C700000000D3
:10E5F0000000000000000000000000000000703873
:10E60000783878387C387E3876387738733873B80D
:10E6100071B871F870F870F8707870380000000008
:10E62000000000000000000000000000000007E003
:10E630001FF83FFC3C3C781E700E700E700E700E82
:10E64000700E781E3C3C3FFC1FF807E00000000005
:10E6500000000000000000000000000000003FE09B
:10E660003FF03FF83878383838783FF83FF03FE0EF
:10E67000380038003800380038003800000000004A
:10E68000000000000000000000000000000007E0A3
:10E690001FF83FFC3C3C781E700E700E700E700E22
:10E6A000708E79DE3CFC3FFC1FFE07EF0006000089
:10E6B00000000000000000000000000000003FE03B
:10E6C0003FF03FF83838383838383FF83FF03FC02F
:10E6D00038E038F0387038383838381C000000001E
:10E6E000000000000000000000000000000007C063
:10E6F0001FF03FF0387838383C001F800FF003F0EF
:10E700000078703878783FF83FF00FC000000000C4
:10E7100000000000000000000000000000007FF08A
:10E720007FF07FF0070007000700070007000700E1
:10E7300007000700070007000700070000000000AF
:10E740000000000000000000000000000000703821
:10E750007038703870387038703870387038703879
:10E760007038703878783FF03FF00FC0000000003C
:10E770000000000000000000000000000000E03881
:10E78000E07870707070707038E038E038E01DC06C
:10E790001DC01DC00F800F800F800700000000000B
:10E7A0000000000000000000000000000000E18701
:10E7B000E187718E718E718E718E399C399C399C76
:10E7C000399C1DB81DB81E781E781E781E78000072
:10E7D0000000000000000000000000000000703891
:10E7E000703838701CE01CE00FC00780078007807D
:10E7F0000FC01CE01CE0387070387038000000005A
:10E800000000000000000000000000000000E038F0
:10E81000E038707038E038E01DC00F800F800700CE
:10E8200007000700070007000700070000000000BE
:10E8300000000000000000000000000000007FF069
:10E840007FF07FF000F001E003C007800F001E00A2
:10E850003C007800F000FFF0FFF0FFF00000000047
:10E8600000000000000000000000000000003E006A
:10E870003E003E00380038003800380038003800CC
:10E8800038003800380038003800380038003E00C2
:10E890003E003E0000000000000000000000C0003C
:10E8A000C000600060006000600030003000300098
:10E8B00038001800180018000C000C0000000000C0
:10E8C0000000000000000000000000000000F80050
:10E8D000F800F800380038003800380038003800F8
:10E8E0003800380038003800380038003800F800A8
:10E8F000F800F80000000000000000000000060022
:10E900000F000F001F80198039C039C070E000006F
:10E9100000000000000000000000000000000000F7
:10E9200000000000000000000000000000000000E7
:10E9300000000000000000000000000000000000D7
:10E9400000000000000000000000000000000000C7
:10E95000FFF0FFF000000000000000000000E000F9
:10E960006000300000000000000000000000000017
:10E970000000000000000000000000000000000097
:10E980000000000000000000000000000000000087
:10E990000000000000001F803FC060E003E01FE0B7
:10E9A0003CE070E070E071E03FE01E7000000000AD
:10E9B00000000000000000000000000000007000E7
:10E9C00070007000700077807FE078E07070707089
:10E9D00070707070707078E07FE0778000000000E9
:10E9E0000000000000000000000000000000000027
:10E9F0000000000000000F003FC039C070E0700050
:10EA00007000700070E039C03FC00F0000000000CF
:10EA10000000000000000000000000000000007086
:10EA20000070007000700F703FF038F07070707000
:10EA300070707070707038F03FF00F700000000060
:10EA400000000000000000000000000000000000C6
:10EA50000000000000000F003FC039C070E07FE000
:10EA60007FE0700070E039C03FC00F000000000080
:10EA7000000000000000000000000000000000F0A6
:10EA800001F0038003803FFC3FFC03800380038090
:10EA90000380038003800380038003800000000064
:10EAA0000000000000000000000000000000000066
:10EAB0000000000000000F703FF038F070707070C0
:10EAC00070707070707038F03FF01F70007070F0F0
:10EAD0007FE01FC000000000000000000000700088
:10EAE00070007000700073C07FE078F0707070701C
:10EAF00070707070707070707070707000000000D6
:10EB00000000000000000000000000000000038082
:10EB100003800000000003800380038003800380E3
:10EB200003800380038003800380038000000000D3
:10EB30000000000000000000000000000000038052
:10EB400003800000000003800380038003800380B3
:10EB5000038003800380038003800380038003809D
:10EB600007000E0000000000000000000000700020
:10EB700070007000700070E071C073807F007F00D3
:10EB80007F007B80718071C070E070E00000000049
:10EB900000000000000000000000000000000380F2
:10EBA000038003800380038003800380038003804D
:10EBB0000380038003800380038003800000000043
:10EBC0000000000000000000000000000000000045
:10EBD00000000000000077CF7FFF71C771C771C7C9
:10EBE00071C771C771C771C771C771C700000000D5
:10EBF0000000000000000000000000000000000015
:10EC000000000000000073C07FE078F0707070704A
:10EC100070707070707070707070707000000000B4
:10EC200000000000000000000000000000000000E4
:10EC30000000000000000F803FE038E0707070704E
:10EC400070707070707038E03FE00F80000000005E
:10EC500000000000000000000000000000000000B4
:10EC600000000000000077807FE078E07070707036
:10EC700070707070707078E07FE077807000700066
:10EC800070007000000000000000000000000000A4
:10EC90000000000000000F703FF038F070707070DE
:10ECA00070707070707038F03FF00F70007000700E
:10ECB0000070007000000000000000000000000074
:10ECC000000000000EFC0FFC03C0038003800380E3
:10ECD0000380038003800380038003800000000022
:10ECE0000000000000000000000000000000000024
:10ECF0000000000000001F803FC070E070007E0038
:10ED00003FC007E000E070E03FC01F80000000004F
:10ED100000000000000000000000000000000000F3
:10ED20000380038003800FF00FF0038003800380D3
:10ED3000038003800380038001F000F000000000E6
:10ED400000000000000000000000000000000000C3
:10ED50000000000000007070707070707070707053
:10ED600070707070707078F03FF01F7000000000DD
:10ED70000000000000000000000000000000000093
:10ED80000000000000007070707038E038E038E07B
:10ED90001DC01DC00F800F8007000700000000008D
:10EDA0000000000000000000000000000000000063
:10EDB000000000000000E38EE38E638C77DC76DCDD
:10EDC00036D836D83EF83C781C701C700000000025
:10EDD0000000000000000000000000000000000033
:10EDE00000000000000070E039C039C01F800F0033
:10EDF0000F000F001F8039C039C070E00000000014
:10EE00000000000000000000000000000000000002
:10EE1000000000000000E0E0E0E071C071C071801F
:10EE20003B803B801B001F001F000E000E001C00DB
:10EE30007C007800000000000000000000000000DE
:10EE40000000000000007FC07FC001C003800700F9
:10EE50000E001C00380070007FC07FC00000000062
:10EE6000000000000000000001000100400223C477
:10EE70000FF01FF81FF8DFFB1FF81FF80FF023C477
:10EE8000400201000100000000000000000000003E
:10EE90000000000000000000000000000000300042
:10EEA00030003000300030003000300030003000E2
:10EEB00030003000300030003000300030003000D2
:10EEC000300030003000000000800080000113C2DC
:10EED00009F000F80078187B007800F809F013C2F8
:10EEE0000001008000800000000000000000000021
:10EEF0000000000000000000000000000000000012
:10EF0000000000000000000000007C20FFE0FFE0A7
:10EF100087C00000000000000000000000000000AA
:10EF2000000000000000008001C003E007F00FF8BF
:10EF30001FFC3FFE7FFF00000000000000000000FB
:10EF40000000000000007FFF3FFE1FFC0FF807F0ED
:10EF500003E001C00080008001C003E007F00FF86B
:10EF60001FFC3FFE7FFF00000000000000000000CB
:10EF70000000000000000000000000000000000091
:10EF80000000000000000000000000000000000081
:10EF90000000000000000000000000000000000071
:10EFA0000000000000007FFF3FFE1FFC0FF807F08D
:10EFB00003E001C00080100B00003FE0202024206F
:10EFC0002220FF202220242020203FE000000000FB
:10EFD000F0EF000800000020EC000000F88E0008B0
:10EFE000DCF00008EC000020742B0000088F000803
:10EFF00000000000010203040102030406070809DF
:10F0000002040608000000000000000000000000EC
:10F0100000000000000000000000000000000000F0
:10F0200000000000000000000000000000000000E0
:10F0300000000000000000000000000000000000D0
:10F0400000000000000000000000000000000000C0
:10F0500000000000000000000000000000000000B0
:10F0600000000000000000000000000000000000A0
:10F07000000000000000000000A24A0400000000A0
:10F080000000000001020304060708090000000058
:10F090000000000000000000000000000000000070
:10F0A000B1AA00081DA7000879AC00087DA60008D9
:10F0B00029A70008D1AA00080000000000000000F5
:10F0C0000000000000000000000000000000000040
:0CF0D00000000000000000000000000034
:04000005080070ED92
:00000001FF
